:1062D900E5467006127AF68F4622E546B40506129F
:1062E9003B738F4622E546B40B061271028F462294
:1062F900E546B40A061268348F4622E546B40F060D
:10630900126C3F8F4622E546B414061264E58F46A7
:1063190022E546B41906127A398F4622E546B41E9B
:1063290006127B0A8F4622E546B42306126C958F26
:106339004622E546B42806127BBF8F4622E546B4BD
:106349002D06127B1E8F4622E546B432051273A331
:036359008F46224A
:107AF600C20890061EE0FFA3E0901CECCFF0A3EFB7
:047B0600F07F0522E5
:103B7300127BBB50477D047F011262515008E53E22
:103B8300B401037F0B227D047F021262515008E5CA
:103B93003EB402037F0B227D047F0312625150085F
:103BA300E53EB403037F0B227D047F041262515070
:103BB30008E53EB404037F0B227F0A227F081275B7
:103BC3008750061253497F00227D057F05126251FB
:103BD3005032901CEEE07002A3E070282046257D51
:103BE300017F011262514003023CE990066CE0FF41
:103BF3007C0A7D701272E8900610E0FFA3E0901C2F
:103C0300EE023CB07D067F051262515031901CF0EC
:103C1300E07002A3E070272048247D017F02126236
:103C2300514003023CE990066DE0FF7C0A7D90124F
:103C330072E8900612E0FFA3E0901CF0806F7D070E
:103C43007F051262515031901CF2E07002A3E070C4
:103C530027204C247D017F031262514003023CE97B
:103C630090066EE0FF7C0A7DB01272E8900614E0C5
:103C7300FFA3E0901CF280357D087F05126251504E
:103C830033901CF4E07002A3E07029204F267D01DD
:103C93007F04126251504F90066FE0FF7C0A7DD083
:103CA3001272E8900616E0FFA3E0901CF4CFF0A395
:103CB300EFF080327D077F06126251500F30290CDE
:103CC300901CECE07002A3E07002C22930380C9023
:103CD3001CECE07002A3E07002C238786CE6B40515
:093CE300057F04125D9D7F05229E
:10710200203842900633E0901D10F0123346E53EDF
:10711200B401062049247F0522E53EB40206204D33
:10712200197F0522E53EB4030620510E7F0522E5B4
:107132003EB404062054037F0522901D10E0D39430
:087142000050C8D2387F0A2278
:10683400E53B700AE53EB40105753B018028E53B64
:10684400700AE53EB40205753B02801AE53B700A06
:10685400E53EB40305753B03800CE53B7008E53E5B
:10686400B40403753B047D077F06126251500C7D0E
:10687400077F06126251501E30291B900650E0FF1C
:106884007C067DF01272E87D017F01126251500690
:09689400120FB3122B647F0F22D6
:106C3F00127BBB503F120FB3202F0920300620319B
:106C4F0003303209E532700512774B800B786CE612
:106C5F00B4050B7F03125D9D122B64120FB3202F0F
:106C6F001020300D20310A203207E5327003122B2D
:106C7F00647F0F2212774B7D057F071262515003FD
:066C8F007F14227F0022A9
:1064E500E4F53B7D077F06126251500C7D077F0660
:1064F500126251505E30295B786CE670047F018032
:1065050008786CE6B404077F02125D9D8038786CCC
:10651500E6B407047601802E7D037F051262515093
:1065250025901CF6E07002A3E0701B900662E0FF68
:106535007C097D301272E8900620E0FFA3E0901CF4
:10654500F6CFF0A3EFF07F0612758750037F002288
:106555007F19227D077F0612625150052029027F8F
:0265650005220D
:107A39007D077F0612625150062029037F05229097
:0A7A49000630E0901D10F07F1E22B1
:107B0A00901D10E070037F2322127BBB50037F0A73
:047B1A00227F1E2286
:106C95007D047F071262515041E53EB4010B900619
:106CA5005EE0FF7C087DB0802EE53EB4020B9006C9
:106CB5005FE0FF7C087DD0801EE53EB4030B9006A7
:106CC50060E0FF7C087DF0800EE53EB4040C900684
:106CD50061E0FF7C097D101272E8900631E0901D9D
:056CE50010F07F2822E1
:037BBF007F2D22F5
:107B1E00901D10E070037F3222127BBB50037F0A50
:047B2E00227F2D2263
:1073A3003058037F32227D047F05126251502890AA
:1073B3001CF8E07002A3E0701E900663E0FF7C09F6
:1073C3007D501272E8900622E0FFA3E0901CF8CFF4
:0C73D300F0A3EFF07F3222C2087F0022FE
:10726500900640E06035D259D224753D031233466D
:10727500122B64120FB3127BBB5009E53D6005125A
:10728500334680F2E4F522F523127BBB4009E53D48
:10729500600512334680F2E53D70D2C259C224C260
:0272A50058226D
:04000E0001000430B9
:030003000269652A
:0B696500C0E0C083C082C0D075D00825
:10697000853082852F83E493FF204404C4540FFFA5
:10698000430FF08F80C284D28500C2870000D28777
:10699000007580FF7580FEC284C28500C28700003A
:1069A0000000D287007580FF30440CC2440530E5FA
:0B69B000307006052F8002D244D2A8F0
:0969BB00D0D0D082D083D0E032AC
:03000B00021BB61F
:101BB600C0E0C0F0C083C082C0D075D008758CD894
:101BC600758A92D28C1242201274ECE531D39400BD
:101BD60040051531021F40753111901D10E0D39458
:101BE600004003E014F0901D11E0D394004003E0A0
:101BF60014F0901D12E0D394004003E014F0901D01
:101C060013E0D394004003E014F0E532D39400408F
:101C16000215321541E541B40A004003021F3D900A
:101C26001C2CF8282873021F40021E91021E59021E
:101C36001E2C021DC2021D58021CEE021C84021C30
:101C460067021C4AD3901CEDE09400901CECE094D3
:101C5600005003021F40A3E024FFF0901CEC021F7B
:101C660031D3901CE9E09400901CE8E09400500306
:101C7600021F40A3E024FFF0901CE8021F317F0101
:101C86001278134003021F40901CE1E09400901C60
:101C9600E0E09400400CA3E024FFF0901CE0E03468
:101CA600FFF0D3901CEFE09400901CEEE09400400F
:101CB6000CA3E024FFF0901CEEE034FFF0D3901C60
:101CC600FBE09400901CFAE094005003021F407D54
:101CD600067F011262514003021F40901CFBE02464
:101CE600FFF0901CFA021F317F02127813400302A4
:101CF6001F40901CE3E09400901CE2E09400400C2E
:101D0600A3E024FFF0901CE2E034FFF0D3901CF136
:101D1600E09400901CF0E09400400CA3E024FFF057
:101D2600901CF0E034FFF0D3901CFDE09400901C72
:101D3600FCE094005003021F407D067F02126251B0
:101D46004003021F40901CFDE024FFF0901CFC02A3
:101D56001F317F031278134003021F40901CE5E0F9
:101D66009400901CE4E09400400CA3E024FFF09063
:101D76001CE4E034FFF0D3901CF3E09400901CF2D6
:101D8600E09400400CA3E024FFF0901CF2E034FF46
:101D9600F0D3901CFFE09400901CFEE094005003EA
:101DA600021F407D067F031262514003021F4090CE
:101DB6001CFFE024FFF0901CFE021F317F04127806
:101DC600134003021F40901CE7E09400901CE6E0DD
:101DD6009400400CA3E024FFF0901CE6E034FFF0F2
:101DE600D3901CF5E09400901CF4E09400400CA302
:101DF600E024FFF0901CF4E034FFF0D3901D01E0E6
:101E06009400901D00E094005003021F407D067F61
:101E1600041262514003021F40901D01E024FFF0AE
:101E2600901D00021F31D3901CEBE09400901CEA39
:101E3600E09400400CA3E024FFF0901CEAE034FF9D
:101E4600F0901D14E0D394005003021F40E014F0FC
:101E5600021F40D3901CF9E09400901CF8E0940017
:101E6600400CA3E024FFF0901CF8E034FFF0D39080
:101E76001CF7E09400901CF6E094005003021F400B
:101E8600A3E024FFF0901CF6021F31786CE6FF7089
:101E960003021F40EFB401059006188027786CE610
:101EA600FFB40219D3901CEBE09400901CEAE09476
:101EB60000403FA3E024FFF0901CEA806EEFB403DD
:101EC6001190061AE0FFA3E0901CEACFF0A3EFF012
:101ED6008020786CE6FFB4041ED3901CEBE09400DF
:101EE600901CEAE09400400AA3E024FFF0901CEA6C
:101EF6008039786C068043EF6405603E786CE6FFB7
:101F0600B4060D901CEA7402F0A37458F006802AF9
:101F1600EFB40726D3901CEBE09400901CEAE09403
:101F260000400EA3E024FFF0901CEAE034FFF080AE
:101F360009786C7600800375410A1279E64008122A
:101F460076194003127A02D0D0D082D083D0F0D056
:021F5600E03277
:030013000261394E
:0D613900C0E0C0F0C083C082C0D075D0109F
:1061460075A0FFC284C285D287C286308018C2A4D9
:10615600C2A5D2A6C2A7E5A0540FF54AD2A7FF1240
:1061660065E7D286804F308118D2A4C2A5D2A6C2D6
:10617600A7E5A0540FF54AD2A7FF12635CD286802A
:1061860034308218C2A4D2A5D2A6C2A7E5A0540F65
:10619600F54AD2A7FF1263DFD2868019308316D262
:1061A600A4D2A5D2A6C2A7E5A0540FF54AD2A7FF4E
:0561B600126462D286B4
:0B61BB00D0D0D082D083D0F0D0E032F2
:106BE800BF0113900632E0901D10F0901D10E0D305
:106BF8009400404280F5BF0213900632E0901D11C8
:106C0800F0901D11E0D39400402C80F5BF03139041
:106C18000632E0901D12F0901D12E0D39400401649
:106C280080F5BF0411900632E0901D13F0901D13FB
:076C3800E0D3940050F722A5
:106CEA00304712205F0F900672E0FF7C0B7D301256
:106CFA0072E8D25F22304B1220610F900673E0FFD8
:106D0A007C0B7D501272E8D26122304E1220620F43
:106D1A00900674E0FF7C0B7D701272E8D26222301A
:106D2A00521120630E900675E0FF7C0B7D90127263
:046D3A00E8D2632216
:1055C900303D1A204617900664E0FF7C097D701271
:1055D90072E8D246C214C210C21CC2182230461444
:1055E900203911900665E0FF7C097D901272E8C2AE
:1055F90046C23D22303E1A204817900666E0FF7CDD
:10560900097DB01272E8D248C215C211C21DC21971
:1056190022304814203A11900667E0FF7C097DD0BA
:105629001272E8C248C23E2230401A204C17900636
:1056390068E0FF7C097DF01272E8D24CC216C212F2
:10564900C21EC21A22304C14203B11900669E0FF99
:105659007C0A7D101272E8C24CC2402230421A20E4
:105669004F1790066AE0FF7C0A7D301272E8D24F2C
:10567900C217C213C21FC21B22304F13203C109005
:10568900066BE0FF7C0A7D501272E8C24FC24222CB
:10517E00124106D28C7F07127587500512001680D9
:10518E00121271927F1F7E0012783A90001FEFF07C
:10519E001276737F08127587500512599280FE9011
:1051AE0006087402F0A37458F090060A7402F0A375
:1051BE007458F090060C7402F0A37458F090060E1A
:1051CE007402F0A37458F0900681E0FF7C0D7D1000
:1051DE001272E8E4FFEFFD3395E0FC74302DF5829A
:1051EE0074003CF583E0FE74F02DF582741A3CF5E4
:1051FE0083EEF00FBF08DED208127A027545017FEA
:10520E0001125D9D900618E0FFA3E0901CEACFF01E
:10521E00A3EFF0C208127A02123346305A11E53E5D
:10522E00B4010C900651E0FF7C077D101272E8125B
:10523E0062D9305B0312444B305C03124338305D4D
:10524E000312488E306003124998124DA77D077FD6
:10525E00061262514002C2291255C9126CEA80B878
:10444B007C007D80C2677F011236B950117F061246
:10445B0075875002D2087F01121F580244EB7C0073
:10446B007D70D2677F011236B95002800D7C007DC2
:10447B0078D2677F011236B950077F01120941804C
:10448B005F7C007DA0D2677F011236B950117D078A
:10449B007F06126251500875450112777480417C7A
:1044AB00007DA8C2677F011236B950197D057F01C7
:1044BB0012625150107F061275875002D2087F018D
:1044CB0012455D801B7C007DB0C2677F011236B93F
:1044DB00500E7F061275875002D2087F01124F973C
:1044EB00E4F54CAF4CEF3395E0FEEF7803C333CEDE
:1044FB0033CED8F92400F58274013EAD82FCD2672D
:10450B007F011236B95038754501AF4CEF3395E04A
:10451B00FE74A02FF58274063EF583E0FFC007AF53
:10452B004CEF3395E0FEEF7805C333CE33CED8F99D
:10453B0024F0F58274103EAD82FCD007126F330568
:10454B004CC3E54C648094A84099C25BC265126D64
:01455B003E21
:01455C00223C
:104338007F061275875002C2087D017F06126251FE
:10434800503D7C007D88C2677F021236B9500BD27F
:10435800097F02121F58C20980257C007D70D26730
:104368007F021236B95002800D7C007D78D2677FBB
:10437800021236B95009D2097F02120941C20990C6
:10438800001FE030E1427C007DA0D2677F02123638
:10439800B950147D077F06126251500B1278607570
:1043A8004502127774801E7C007DA8C2677F0212C6
:1043B80036B950147D057F02126251500B12786095
:1043C8007F0212455D1279517D027F0612625150BB
:1043D8006AE4F54CAF4CEF3395E0FEEF7803C33356
:1043E800CE33CED8F92400F58274013EAD82FCD2DA
:1043F800677F021236B95038754502AF4CEF3395D6
:10440800E0FE74A02FF58274063EF583E0FFC00736
:10441800AF4CEF3395E0FEEF7805C333CE33CED8FB
:10442800F924F0F58274103EAD82FCD007126F3388
:10443800054CC3E54C648094A84099C25CC26612DE
:024448006D9273
:01444A00224F
:10488E007D037F06126251503D7C007D90C2677F92
:10489E00031236B9500BD20E7F03121F58C20E8070
:1048AE00257C007D70D2677F031236B95002800DD1
:1048BE007C007D78D2677F031236B95009D20E7F05
:1048CE0003120941C20E90001FE030E2427C007DCF
:1048DE00A0D2677F031236B950147D077F0612628D
:1048EE0051500B127860754503127774801E7C0050
:1048FE007DA8C2677F031236B950147D057F03125F
:10490E006251500B1278607F0312455D1279517D12
:10491E00047F06126251506AE4F54CAF4CEF3395AA
:10492E00E0FEEF7803C333CE33CED8F92400F58200
:10493E0074013EAD82FCD2677F031236B9503875D2
:10494E004503AF4CEF3395E0FE74A02FF58274064D
:10495E003EF583E0FFC007AF4CEF3395E0FEEF78F6
:10496E0005C333CE33CED8F924F0F58274103EADA4
:10497E0082FCD007126F33054CC3E54C648094A8BB
:09498E004099C25DC228126DE6D9
:0149970022FD
:104998007D057F06126251503D7C007D98C2677F7D
:1049A800041236B9500BD20C7F04121F58C20C8067
:1049B800257C007D70D2677F041236B95002800DC5
:1049C8007C007D78D2677F041236B95009D20C7FFB
:1049D80004120941C20C90001FE030E3427C007DC4
:1049E800A0D2677F041236B950147D077F06126281
:1049F80051500B127860754504127774801E7C0044
:104A08007DA8C2677F041236B950147D057F041251
:104A18006251500B1278607F0412455D1279517D06
:104A2800067F06126251506AE4F54CAF4CEF33959D
:104A3800E0FEEF7803C333CE33CED8F92400F582F5
:104A480074013EAD82FCD2677F041236B9503875C6
:104A58004504AF4CEF3395E0FE74A02FF582740641
:104A68003EF583E0FFC007AF4CEF3395E0FEEF78EB
:104A780005C333CE33CED8F924F0F58274103EAD99
:104A880082FCD007126F33054CC3E54C648094A8B0
:094A98004099C260C22A126E3A74
:014AA10022F2
:106FD300BF010AC214C210C21CC2188025BF020A14
:106FE300C215C211C21DC2198018BF030AC216C23C
:106FF30012C21EC21A800BBF0408C217C213C21FDB
:10700300C21B90001FE0FF30E002D224EF30E10208
:0E701300D225EF30E202D226EF30E302D22780
:01702100224C
:1065E7008F4B7868E6C39450507130496E20596BD1
:1065F7007D077F01126251502B205E287868E67074
:106607000D90063BE0B54B06203F03D23F22202FDB
:106617000D203F0A7F01126FD3753D02D22F9006DE
:1066270034E0F5327D087F06126251501990063F1B
:10663700E0B54B06205E03D265220534E534AE3360
:10664700700E0533800A0534E534AE337002053326
:0C66570014F5828E83E54BF07868062273
:10635C008F4B7869E6C394505078304D7520597244
:10636C007D077F0212625150327F02127813502B3C
:10637C00205E287869E6700D90063BE0B54B062050
:10638C004103D2412220300D20410A7F02126FD3EB
:10639C00753D02D230900634E0F5327D087F06124E
:1063AC006251501990063FE0B54B06205E03D26651
:1063BC00220536E536AE35700E0535800A0536E514
:1063CC0036AE357002053514F5828E83E54BF078C8
:0363DC006906222D
:1063DF008F4B786AE6C394505078305175205972BC
:1063EF007D077F0312625150327F03127813502BB7
:1063FF00205E28786AE6700D90063BE0B54B0620CC
:10640F004303D2432220310D20430A7F03126FD35F
:10641F00753D02D231900634E0F5327D087F0612C9
:10642F006251501990063FE0B54B06205E03D2280B
:10643F00220538E538AE37700E0537800A0538E586
:10644F0038AE377002053714F5828E83E54BF0783E
:03645F006A0622A8
:106462008F4B786BE6C39450507830547520597234
:106472007D077F0412625150327F04127813502B31
:10648200205E28786BE6700D90063BE0B54B062047
:106492004503D2452220320D20450A7F04126FD3D4
:1064A200753D02D232900634E0F5327D087F061245
:1064B2006251501990063FE0B54B06205E03D22A86
:1064C20022053AE53AAE39700E0539800A053AE5F9
:1064D2003AAE397002053914F5828E83E54BF078B5
:0364E2006B062224
:1078600090001FE0FF30E004D208D220EF30E104A6
:10787000D209D221EF30E204D20ED222EF30E3045B
:05788000D20CD223220E
:10795100C220C221C222C22390001FE0FF30E102F7
:0F796100C209EF30E202C20EEF30E302C20C2285
:105D9D008F4C304603025E39304803025E39304C79
:105DAD0003025E39304F03025E397D017F011262BD
:105DBD00515079E54CB401197D017F0512625150A6
:105DCD000C90065AE0FF7C087D301272E8786C0664
:105DDD0022E54CB402177D027F05126251504890A6
:105DED00065BE0FF7C087D501272E8803AE54CB40A
:105DFD00041A7D027F05126251500C90065DE0FF82
:105E0D007C087D901272E8786C760622E54C64036E
:105E1D00701E7D027F05126251500C90065CE0FFF2
:105E2D007C087D701272E8786C760122E4786CF64D
:015E3D002242
:107A1E00EF1FAA0670011ED39400EA9400400BE4F7
:0A7A2E00FDEDC394C850E90D80F788
:017A3800222B
:105A47008F5D306B5BE55DB40111D22090001FE0E4
:105A5700F420E003305E44D2088040E55DB40211D3
:105A6700D22190001FE0F420E103305E2ED209809E
:105A77002AE55DB40311D22290001FE0F420E2036F
:105A8700305E18D20E8014E55DB4040FD223900067
:105A97001FE0F420E303305E02D20CAF5D026BE837
:105AA700E55DB40110C22090001FE0F420E0033050
:105AB7005E41C20822E55DB40210C22190001FE0DA
:105AC700F420E103305E2CC20922E55DB40310C265
:105AD7002290001FE0F420E203305E17C20E22E599
:105AE7005DB4040FC22390001FE0F420E303305E8F
:045AF70002C20C22B9
:105AFB008F5330695BE553B40111D22490001FE042
:105B0B00F420E003305E44D2088040E553B4021128
:105B1B00D22590001FE0F420E103305E2ED20980E5
:105B2B002AE553B40311D22690001FE0F420E203C0
:105B3B00305E18D20E8014E553B4040FD2279000B8
:105B4B001FE0F420E303305E02D20CAF53026BE88C
:105B5B00E553B40110C22490001FE0F420E00330A1
:105B6B005E41C20822E553B40210C22590001FE02B
:105B7B00F420E103305E2CC20922E553B40310C2BA
:105B8B002690001FE0F420E203305E17C20E22E5E0
:105B9B0053B4040FC22790001FE0F420E303305EE0
:045BAB0002C20C2204
:08290E008F538C548D558B563C
:10291600C267E55524FFF582E55434FFF583E0F5FB
:1029260058855582855483E0FFF559A3E0FEF55A94
:10293600EF14B40800505C90294B75F003A4C583CE
:1029460025F0C5837302296302296A0229710229C7
:102956007802297F02298602298D0229947557015A
:10296600D267802F755702D2678028755704D267C1
:102976008021755708D267801A755710D267801361
:10298600755720D267800C755740D26780057557FA
:1029960080D267EE24FE7003022A5B24F8605C2472
:1029A600096003022A6DE553B401059000208045B5
:1029B600E553B40205900021803BE553B40305902E
:1029C60000228031E553B404059000238027E553A7
:1029D600B40505900024801DE553B4060590002536
:1029E6008013E553B407059000268009E553640873
:1029F6007077900027E04557F0806EE553B40105E7
:102A06009000208045E553B40205900021803BE507
:102A160053B403059000228031E553B404059000B9
:102A2600238027E553B40505900024801DE553B4A3
:102A360006059000258013E553B40705900026800F
:102A460009E55364087022900027E0FFE557F4FE7D
:102A5600EF5EF08014E553B4080D855582855483E6
:102A6600E0FF1260A5C267C267206703022B63E519
:102A760053B40109900020E0FD7F208060E553B447
:102A86000209900021E0FD7F218052E553B403093D
:102A9600900022E0FD7F228044E553B404099000B3
:102AA60023E0FD7F238036E553B40509900024E03A
:102AB600FD7F248028E553B40609900025E0FD7FBC
:102AC60025801AE553B40709900026E0FD7F26808D
:102AD6000CE553B4080C900027E0FD7F277E00121A
:102AE6007328D2AFD26BAF56125A47AD58E4FF12D5
:102AF60076F7AD59E4FF1276F7E55AB401047D384E
:102B06008007E55AB40A077D367F061276F7E55345
:102B1600B408031276737D077F06126251500B20AC
:102B26002908C208C209C20EC20C7D017F011262C9
:102B3600514002C2087D017F021262514002C20961
:102B46007D017F031262514002C20E7D017F041295
:0D2B560062514002C20CC26BAF56125A47CA
:012B6300224F
:045E3E008F538D549D
:105E4200D26BAF54125A47AF54126BE8E553B40108
:105E5200059000208044E553B40205900021803A69
:105E6200E553B403059000228030E553B404059055
:105E720000238026E553B40505900024801CE553D9
:105E8200B406059000258012E553B407059000265C
:105E92008008E553B40806900027E0F555E5556003
:105EA20025755701E4F556E55530E007AD57E4FF97
:105EB2001276F7E555C313F55505570556E556C352
:105EC200940840E3800E7D187F021276F77D537F9F
:0B5ED200021276F7C26BAF54125A4761
:015EDD0022A2
:021F58008F4DAB
:101F5A00E54D6401701E754E1B754F10900080E0B0
:101F6A00F550E54F2550F582E4354EF583E0F552FC
:101F7A0078688069E54D6402701E754E1B754F6066
:101F8A00900088E0F550E54F2550F582E4354EF58E
:101F9A0083E0F55278698045E54D6403701E754EFD
:101FAA001B754FB0900090E0F550E54F2550F58233
:101FBA00E4354EF583E0F552786A8021E54DB404A4
:101FCA001F754E1C754F00900098E0F550E54F259F
:101FDA0050F582E4354EF583E0F552786BE6F5511B
:101FEA00E55214B4090040030222F790200375F069
:101FFA0003A4C58325F0C5837302201E0220710243
:10200A0020C402211702216A0221BD0222100222E3
:10201A00610222B1E54F2550F582E4354EF583A3DE
:10202A00E0B40A18E5502402FFE433FEE551B5078F
:10203A000BE4B50607AD4D7F01022286AF507E0044
:10204A00EF2403FDEE33FCE5516D7001EC600302F1
:10205A0022F7EF254FFFEE354ECF2401FDE43FFC7A
:10206A00AB4D7F010222AEE54F2550F582E4354E95
:10207A00F583A3E0B40A18E5502402FFE433FEE531
:10208A0051B5070BE4B50607AD4D7F02022286AFB4
:10209A00507E00EF2403FDEE33FCE5516D7001EC38
:1020AA0060030222F7EF254FFFEE354ECF2401FDE4
:1020BA00E43FFCAB4D7F020222AEE54F2550F5828C
:1020CA00E4354EF583A3E0B40A18E5502402FFE490
:1020DA0033FEE551B5070BE4B50607AD4D7F0302A4
:1020EA002286AF507E00EF2403FDEE33FCE5516DEE
:1020FA007001EC60030222F7EF254FFFEE354ECF59
:10210A002401FDE43FFCAB4D7F030222AEE54F25DF
:10211A0050F582E4354EF583A3E0B40A18E550245D
:10212A0002FFE433FEE551B5070BE4B50607AD4DF2
:10213A007F04022286AF507E00EF2403FDEE33FCBB
:10214A00E5516D7001EC60030222F7EF254FFFEEB7
:10215A00354ECF2401FDE43FFCAB4D7F040222AE95
:10216A00E54F2550F582E4354EF583A3E0B40A180D
:10217A00E5502402FFE433FEE551B5070BE4B5064A
:10218A0007AD4D7F05022286AF507E00EF2403FD86
:10219A00EE33FCE5516D7001EC60030222F7EF2586
:1021AA004FFFEE354ECF2401FDE43FFCAB4D7F05DA
:1021BA000222AEE54F2550F582E4354EF583A3E0C1
:1021CA00B40A18E5502402FFE433FEE551B5070BC3
:1021DA00E4B50607AD4D7F06022286AF507E00EFBA
:1021EA002403FDEE33FCE5516D7001EC600302221D
:1021FA00F7EF254FFFEE354ECF2401FDE43FFCAB50
:10220A004D7F060222AEE54F2550F582E4354EF5A4
:10221A0083A3E0B40A17E5502402FFE433FEE55134
:10222A00B5070AE4B50606AD4D7F07804FAF507E6D
:10223A0000EF2403FDEE33FCE5516D7001EC600301
:10224A000222F7EF254FFFEE354ECF2401FDE43F82
:10225A00FCAB4D7F07804DE54F2550F582E4354EA6
:10226A00F583A3E0B40A18E5502402FFE433FEE53F
:10227A0051B5070BE4B50607AD4D7F08025E3EAFC8
:10228A00507E00EF2403FDEE33FCE5516D7001EC46
:10229A00705BEF254FFFEE354ECF2401FDE43FFC86
:1022AA00AB4D7F0802290EE54F2550F582E4354EE5
:1022BA00F583A3A3E07036E54F2550F582E4354E49
:1022CA00F583A3E024F96008147022AF4D0277EC7D
:1022DA00D26B7F01125A47AF4D126BE87D5E7F02C7
:0D22EA001276F7C26B7F01125A471259920B
:0122F70022C4
:0436B9008C4D8D4E59
:1036BD00054EE54E7002054D14F5828C83E0F970D0
:1036CD000302385BBF010875331B753410801FBFB3
:1036DD00020875351B7536608014BF030875371BDE
:1036ED007538B08009BF040675391C753A0020671E
:1036FD00030237C1BF01087868E6696002C322BFC3
:10370D0002087869E6696002C322BF0308786AE699
:10371D00696002C322BF0408786BE6696002C322A8
:10372D00E4FEEEC39940030237BFEF6401701CE560
:10373D004E2EF582E4354DF583E0FDE5342EF58210
:10374D00E43533F583E06D6002C322EF6402701C33
:10375D00E54E2EF582E4354DF583E0FDE5362EF58B
:10376D0082E43535F583E06D6002C322EF640370AA
:10377D001CE54E2EF582E4354DF583E0FDE5382E42
:10378D00F582E43537F583E06D6002C322EF640402
:10379D00701CE54E2EF582E4354DF583E0FDE53ADE
:1037AD002EF582E43539F583E06D6002C3220E02F9
:1037BD00372FD32230670302385CE4FEEEC3994005
:1037CD0003023859EF6401701CE54E2EF582E43585
:1037DD004DF583E0FDE5342EF582E43533F583E0D8
:1037ED006D6065C322EF6402701CE54E2EF582E418
:1037FD00354DF583E0FDE5362EF582E43535F5835F
:10380D00E06D6044C322EF6403701CE54E2EF5821B
:10381D00E4354DF583E0FDE5382EF582E43537F5D9
:10382D0083E06D6023C322EF6404701CE54E2EF51A
:10383D0082E4354DF583E0FDE53A2EF582E4353928
:0F384D00F583E06D6002C3220E0237C9D322C398
:01385C002249
:102B640090001FE0540FF55CB4010BE53EB4010383
:102B7400D21422C21422E55C6403702AE53EB40137
:102B840006D214D2108004C214C210E53EB402115D
:102B9400D2157D017F071262514003022D7FD211AD
:102BA40022C215C21122E55C6405702AE53EB40117
:102BB40006D214D21C8004C214C21CE53EB4031114
:102BC400D2167D027F071262514003022D7FD21E6E
:102BD40022C216C21E22E55C6409702AE53EB401D5
:102BE40006D214D2188004C214C218E53EB40411EB
:102BF400D2177D037F071262514003022D7FD21B3F
:102C040022C217C21B22E55C6407704EE53EB40184
:102C140008D214D210D21C8006C214C210C21CE501
:102C24003EB40211D2157D017F071262515002D2C7
:102C340011D21D8006C215C211C21DE53EB4031394
:102C4400D216D2127D027F071262514003022D7FF9
:102C5400D21E22C216C212C21E22E55C640B704E42
:102C6400E53EB40108D214D210D2188006C214C2B0
:102C740010C218E53EB40211D2157D017F0712621D
:102C8400515002D211D2198006C215C211C219E5DF
:102C94003EB40413D217D2137D037F07126251404E
:102CA40003022D7FD21B22C217C213C21B22E55C72
:102CB400640D704BE53EB40108D214D21CD21880C6
:102CC40006C214C21CC218E53EB40311D2167D021A
:102CD4007F071262515002D21ED21A8006C216C257
:102CE4001EC21AE53EB40413D217D21F7D037F0718
:102CF4001262514003022D7FD21B22C2178078E555
:102D04005C640F7076E53EB4010AD214D210D21C72
:102D1400D2188008C214C210C21CC218E53EB40204
:102D240013D2157D017F071262515002D211D21DB8
:102D3400D2198008C215C211C21DC219E53EB403DE
:102D440013D216D2127D027F071262515002D21E94
:102D5400D21A8008C216C212C21EC21AE53EB404B8
:102D640012D217D213D21F7D037F07126251500B68
:0B2D7400D21B22C217C213C21FC21BD9
:012D7F002231
:100FB30090001FE0540FF55CB401167D017F011210
:100FC3006251500A7F061275874003D20822C20875
:100FD30022E55C6403705BE53E640170257D017F5F
:100FE30001126251500B7F061275874004D20880AC
:100FF30002C2087D017F021262515003D20922C24C
:101003000922E53E640260030214637D017F01123D
:1010130062515004D2088002C2087D017F0212622D
:1010230051500C7D017F071262515003D20922C235
:101033000922E55C6405705BE53E640170257D0172
:101043007F01126251500B7F061275874004D2084C
:101053008002C2087D017F031262515003D20E2227
:10106300C20E22E53E640360030214637D017F0127
:101073001262515004D2088002C2087D017F03121C
:101083006251500C7D027F071262515003D20E222F
:10109300C20E22E55C6409705BE53E640170257D48
:1010A300017F01126251500B7F061275874004D2F3
:1010B300088002C2087D017F041262515003D20CE2
:1010C30022C20C22E53E640460030214637D017FA7
:1010D300011262515004D2088002C2087D017F04CC
:1010E300126251500C7D037F071262515003D20CE0
:1010F30022C20C22E55C640760030211B5E53E647D
:101103000170347D017F01126251500B7F0612750D
:10111300874004D2088002C2087D017F0212625117
:101123005004D2098002C2097D017F03126251502B
:1011330003D20E22C20E22E53E640270367D017F89
:10114300011262515004D2088002C2087D017F025D
:10115300126251500D7D017F071262515004D20972
:101163008002C2097D017F031262515003D20E2215
:10117300C20E22E53E640360030214637D017F0116
:101183001262515004D2088002C2087D017F02120C
:1011930062515004D2098002C2097D017F031262A9
:1011A30051500C7D027F071262515003D20E22C2AE
:1011B3000E22E55C640B6003021273E53E6401706A
:1011C300347D017F01126251500B7F0612758740F7
:1011D30004D2088002C2087D017F021262515004CA
:1011E300D2098002C2097D017F041262515003D2E9
:1011F3000C22C20C22E53E640270367D017F01128F
:1012030062515004D2088002C2087D017F0212623B
:1012130051500D7D017F071262515004D2098002A3
:10122300C2097D017F041262515003D20C22C20C09
:1012330022E53E640460030214637D017F011262B0
:10124300515004D2088002C2087D017F021262510C
:101253005004D2098002C2097D017F0412625150F9
:101263000C7D037F071262515003D20C22C20C2261
:10127300E55C640D6003021331E53E640170347D67
:10128300017F01126251500B7F061275874004D211
:10129300088002C2087D017F031262515004D20EFE
:1012A3008002C20E7D017F041262515003D20C22D0
:1012B300C20C22E53E640370367D017F0112625148
:1012C3005004D2088002C2087D017F03126251508C
:1012D3000D7D027F071262515004D20E8002C20EAE
:1012E3007D017F041262515003D20C22C20C22E50D
:1012F3003E640460030214637D017F011262515056
:1013030004D2088002C2087D017F03126251500497
:10131300D20E8002C20E7D017F04126251500C7DF9
:10132300037F071262515003D20C22C20C22E55CE8
:10133300640F6003021463E53E640170437D017F23
:1013430001126251500B7F061275874004D2088048
:1013530002C2087D017F021262515004D209800249
:10136300C2097D017F031262515004D20E8002C272
:101373000E7D017F041262515003D20C22C20C2253
:10138300E53E640270457D017F011262515004D233
:10139300088002C2087D017F02126251500D7D0157
:1013A3007F071262515004D2098002C2097D017F76
:1013B300031262515004D20E8002C20E7D017F04DB
:1013C3001262515003D20C22C20C22E53E64037018
:1013D300457D017F011262515004D2088002C20888
:1013E3007D017F021262515004D2098002C2097D3D
:1013F300017F03126251500D7D027F07126251502B
:1014030004D20E8002C20E7D017F0412625150038A
:10141300D20C22C20C22E53E640470447D017F019C
:101423001262515004D2088002C2087D017F021269
:1014330062515004D2098002C2097D017F03126206
:10144300515004D20E8002C20E7D017F04126251FC
:10145300500C7D037F071262515003D20C22C20C41
:011463002266
:1078F0007F011278135010C209C20EC20C7F06120B
:107900007587500CC208227F011278134002C2080A
:017910002254
:107A6D007F021278135007C209C20EC20C227F0288
:087A7D001278134002C2092235
:107A85007F031278135007C209C20EC20C227F036E
:087A95001278134002C20E2218
:107A9D007F041278135007C209C20EC20C227F0454
:087AAD001278134002C20C2202
:1069C4000500050105030507050F051F051E051C28
:1069D400051805100201040E040A03060101040B44
:1069E4000304040F020304010302040D0200020263
:1069F4000300040904040305030701000303040757
:106A0400030104060402040C05160515000006150E
:0E6A1400062A060C06380633061E0612061762
:10526E00203737900640E004F519D36480948150BE
:10527E0003025348D3E5196480948F400375190FC8
:10528E0090063DE0FF123E6090063EE0F518E4F514
:10529E001ED237C264C257C24A22304A60306416E8
:1052AE00152EE52ED394004003025348C2CAC264A1
:1052BE00D25785182E2230570E152EE52ED3940078
:1052CE005078C264C25722AF1C151CEF700BC24A35
:1052DE00E51825E0F52ED25722E51D30E00585189C
:1052EE002E8008E51875F003A4F52EAF1D7801EF9A
:1052FE0008800103D8FDF51DD264D2CA22D5190843
:10530E00C237E4F53DC25822051E7440251EF582B3
:10531E00E43406F583E025E024C4F582E43469F52F
:10532E0083E493540FF51C740193F51D700AD25744
:0A533E00E51825E025E0F52ED24A1F
:015348002242
:105F770020371A90063DE0FF123E6090063EE0F59E
:105F87001AE4F51ED237C264C257C24A22304A59B0
:105F9700306413152EE52ED39400506BC2CAC26429
:105FA700D257851A2E2230570E152EE52ED3940080
:105FB7005055C264C25722AF1C151CEF7007C24A66
:105FC700C237F53D22E51D30E005851A2E8008E52C
:105FD7001A75F003A4F52EAF1D7801EF08800103B1
:105FE700D8FDF51DD264D2CA22E53F25E024C4F5C9
:105FF70082E43469F583E493FA740193FBEA540F5E
:07600700F51CEBF51DD24A68
:01600E00226F
:107B3200C3EF648094A15008EF25E025E0F52E22E2
:047B4200E4F52E2216
:1074B800BF010790063E7418F022BF020790063EEF
:1074C8007412F022BF030590063E8014BF04079093
:1074D800063E740BF02290063EBF05047409F022A4
:0474E800740CF0220E
:103E6000EF14B420004003023FB3903E7875F00396
:103E7000A4C58325F0C58373023ED8023EDF023E0F
:103E8000E6023EED023EF4023EFB023F02023F0923
:103E9000023F10023F17023F1E023F25023F2C0245
:103EA0003F33023F3A023F41023F48023F4F023F49
:103EB00056023F5D023F64023F6B023F72023F7950
:103EC000023F80023F87023F8E023F95023F9702EA
:103ED0003F9E023FA5023FAC75CB8E75CAC62275C8
:103EE000CB9575CA772275CB9B75CA692275CBA015
:103EF00075CABA2275CBA675CA332275CBAB75CA03
:103F0000632275CBB075CA022275CBB475CAA322E1
:103F100075CBB875CAFA2275CBBC75CAD82275CBD9
:103F2000C075CAA82275CBC475CA362275CBC775B1
:103F3000CA862275CBCA75CABC2275CBCD75CAB4E8
:103F40002275CBD075CA762275CBD375CA3022754F
:103F5000CBD575CAB22275CBD875CA132275CBDA08
:103F600075CA522275CBDC75CA7D2275CBDD75CA48
:103F70006E2275CBE075CA542275CBE275CA1B223E
:103F800075CBE375CAC32275CBE575CA5E2275CBC6
:103F9000E675CADA22801C75CBE875CA902275CB0B
:103FA000EA75CAD92275CBEC75CA092275CBED75B5
:0A3FB000CA292275CBE875CA412228
:1071DA00EFC39400403FEF9408503AE4FEEF75F095
:1071EA0008A42430F582E43400F583E5822EF58282
:1071FA00E43583F583E0FCED75F008A424E8F58214
:10720A00E4341AF583E5822EF582E43583F583ECBE
:05721A00F00EBE08C8E3
:01721F00224C
:1060A5008F5BE55B6405701D200A0DD20A7FF47EC7
:1060B50001127A1EC20A8074C20A7FF47E01127A26
:1060C5001ED20A8067E55B6406701D200B0DD20B9E
:1060D5007FF47E01127A1EC20B800BC20B7FF47E09
:1060E50001127A1ED20B8044E55B6407701D200FF8
:1060F5000DD20F7FF47E01127A1EC20F800BC20FE4
:106105007FF47E01127A1ED20F8021E55B64087050
:1061150022200D0DD20D7FF47E01127A1EC20D8054
:106125000BC20D7FF47E01127A1ED20D7FF47E0123
:04613500127A1E229A
:104DA700A233B330B401B350357D017F081262518D
:104DB7005027A233B35010A2B4B3500B900652E061
:104DC700FF7C077D30800F30330F30B40C900653D3
:104DD700E0FF7C077D501272E8A2B4B39233A2348D
:104DE700B330B501B350357D027F081262515027A9
:104DF700A234B35010A2B5B3500B900654E0FF7C19
:104E0700077D70800F30340F30B50C900655E0FFEA
:104E17007C077D901272E8A2B5B39234A235B33005
:104E2700B701B350357D037F081262515027A23571
:104E3700B35010A2B7B3500B900656E0FF7C077D26
:104E4700B0800F30350F30B70C900657E0FF7C0766
:104E57007DD01272E8A2B7B39235A236B330B6014D
:104E6700B350357D047F081262515027A236B350E4
:104E770010A2B6B3500B900658E0FF7C077DF08078
:104E87000F30360F30B60C900659E0FF7C087D10C6
:094E97001272E8A2B6B3923622B1
:10767300900027E0FF30E404D20A8002C20AEF3010
:10768300E504D20B8002C20BEF30E604D20F800276
:0B769300C20FEF30E703D20D22C20D42
:01769E0022C9
:1074180090063CE0FF602E20370F6029123E60D2B4
:10742800CAD237D264752E1422E52ED394004003B5
:10743800152E22206408D2CA752E14D26422C2CA1C
:06744800752E7DC26422D6
:10744E002037127F1C123E60D2CAD237D264752EFC
:10745E0064751B3C22E52ED394004003152E22AFFB
:10746E001B151BD3EF648094804004752E6422C2DA
:04747E0037E4F53DBD
:0174820022E7
:104EA00020371C754006E53E75F008A424E8F5821D
:104EB000E4341AF583E06003D23722E4F53D22E5BD
:104EC0002ED394004003152E22C2CA1540E540148B
:104ED0007003024F5B14606F14604014602E146006
:104EE00003024F8FE53E75F008A424E8F582E43410
:104EF0001AF583E0FF7003F53D22123E60E53E7532
:104F0000F008A424E9F582E4341A8079E53E75F0CE
:104F100008A424EAF582E4341A80397408441B702A
:104F200003F53D22E53E75F008A424EBF582E43458
:104F30001AF583E0FF123E60E53E75F008A424EC0C
:104F4000F582E4341A803EE53E75F008A424EDF5C0
:104F500082E4341AF583E0FF027B327420441B7034
:104F600003F53D22E53E75F008A424EEF582E43415
:104F70001AF583E0FF123E60E53E75F008A424EFC9
:104F8000F582E4341AF583E0FF127B32D2CA22E4C0
:074F9000F53DC2CAC2372241
:1074EC00E53D14601C14601C14601C14601F1460B7
:1074FC001F2405701EC2CAC237C264C257E4F540CD
:10750C0022024EA002741812526ED2582202744EED
:04751C00125F772261
:10761900E52365437004E5226542601F85224285A2
:107629002343C2A4D2A5C2A6C2A700AF23127ACB14
:0D763900E522FF127ACB00D2A7D322C32294
:1079E600E52465446014852444D2A4D2A5C2A6C267
:0C79F600A7AF24127ACBD2A7D322C32261
:107A0200E521653C601485213CD2A4C2A5C2A6C270
:0C7A1200A7AF21127ACBD2A7D322C32247
:10410600E4F54CF54D754E1E754FFF854D82854C79
:1041160083E0F5506350FFE550F0E0655060031210
:104126007BC26350FF854D82854C83E550F0E06588
:10413600506003127BC2054DE54D7002054CE54FFC
:10414600154F7002154ED3E54F9400E54E9400507E
:10415600BAE4F54CF54DF54EF54FE54D254FF58294
:10416600E54C354EF583E4F0054FE54F7002054EFC
:10417600B4FFE7E54EB41EE275985A758921758835
:1041860045758845758DE775878075C90275331B3A
:1041960075341075351B75366075371B7538B075F7
:1041A600391C753A0075B701D2A9D2A8D2AA9006D1
:1041B60000E0FFA3E0901CE0CFF0A3EFF090060232
:1041C600E0FFA3E0901CE2CFF0A3EFF0900604E03E
:1041D600FFA3E0901CE4CFF0A3EFF0900606E0FF0B
:1041E600A3E0901CE6CFF0A3EFF0901CFA7417F052
:1041F600A37499F0901CFC7417F0A37499F0901CAA
:10420600FE7417F0A37499F0901D007417F0A37450
:0942160099F0D291D2AF12772188
:01421F00227C
:027BC20080FE43
:10758700C2AFC284D285BF060AC286E580A2E19255
:107597006B8018BF070AC286E580A2E2926B800B58
:1075A700BF0808C286E580A2E3926BD286D2AFA25B
:0175B7006B68
:0175B80022B0
:10625100BF0107900020E0FE8048BF0207900021A7
:10626100E0FE803EBF0307900022E0FE8034BF04C1
:1062710007900023E0FE802ABF0507900024E0FE7E
:106281008020BF0607900025E0FE8016BF0707901B
:106291000026E0FE800CBF0807900027E0FE800288
:1062A100E4FEBD0103EE1322BD0204EEA2E122BD14
:1062B1000304EEA2E222BD0404EEA2E322BD050422
:1062C100EEA2E422BD0604EEA2E522BD0704EEA281
:0762D100E622BD0802EE33D6
:0162D80022A3
:024F97008F4D3C
:104F99009000B0E0F54EE54D64017037E54E24020E
:104FA900FFE433FE7868E66F7001EE600302508C0F
:104FB9007410254EF582E4341BAF82F5508F51D21F
:104FC9006B7F01125A471279AC12385DC26B7F01AF
:104FD900025089E54D64027037E54E2402FFE4333F
:104FE900FE7869E66F7001EE600302508C746025EB
:104FF9004EF582E4341BAF82F5508F51D26B7F029C
:10500900125A471279AC12385DC26B7F020250897D
:10501900E54D64037033E54E2402FFE433FE786AFC
:10502900E66F7001EE705C74B0254EF582E4341BB6
:10503900AF82F5508F51D26B7F03125A471279AC68
:1050490012385DC26B7F038037E54D64047034E527
:105059004E2402FFE433FE786BE66F7001EE702395
:105069007400254EF582E4341CAF82F5508F51D27D
:105079006B7F04125A471279AC12385DC26B7F04F8
:03508900125A4771
:01508C002201
:04385D008F4FE4FDA8
:023861008D5781
:1038630075F020EFA42460F582E5F03403AF82F510
:103873005A8F5BF583E0F558D3940050030239E97E
:10388300E558941040030239E9E557704C7FF47E04
:1038930001127A1EE55825E0F558755901E55824BB
:1038A30001FFE433FEC3E5599FEE6480F87480980A
:1038B30040030239E9E55B2559F582E4355AF5837E
:1038C300E0FFE55B2559F582E4355AF583A3E0FD76
:1038D3001276F70559055980C4E5576401707AC219
:1038E3002B7FF47E01127A1EE55825E0F5587559B1
:1038F30001E5582401FFE433FEC3E5599FEE6480DC
:10390300F874809840030239E9E55B2559F582E4B0
:10391300355AF583E0FFE55B2559F582E4355AF521
:1039230083A3E0FD1276F790001FE0FF30E006303E
:103933004903C22022EF30E106304D03C22122EFBA
:1039430030E206305103C22222EF30E30630540343
:10395300C22322055905598098E557640260030282
:1039630039E9C22BC22CC22DC22E7FF47E01127AFA
:103973001EE55825E0F558755901E5582401FFE483
:1039830033FEC3E5599FEE6480F87480985057E581
:103993005B2559F582E4355AF583E0FFE55B25594C
:1039A300F582E4355AF583A3E0FD1276F790001F04
:1039B300E030E005303902802290001FE030E1055D
:1039C300303A02801690001FE030E205303B02805F
:1039D3000A90001FE030E308303C05C22002726504
:0639E3000559055980940E
:0139E90022BB
:02455D008F4D80
:10455F00C2679000A8E0FFE54DB401167868E6FE4B
:10456F00D39F400EEE9FF55074102FF582E4341B4D
:10457F00804FE54DB402167869E6FED39F400EEEEC
:10458F009FF55074602FF582E4341B8034E54DB4F1
:10459F000316786AE6FED39F400EEE9FF55074B077
:1045AF002FF582E4341B8019E54DB4041C786BE6BB
:1045BF00FED39F4014EE9FF55074002FF582E43424
:1045CF001CAF82F5518F52D26720670302466DD21E
:1045DF006BAF4D125A477FF47E01127A1E7D207FFA
:1045EF00051276F77D1A7F081276F77FC87E0012C4
:1045FF007A1EE4F54EE54EC39550505B0552E552D9
:10460F00AE517002055114F5828E83E0F54F60367E
:10461F0024F5601414601714601A14601D146020C0
:10462F0024057028E4FD80277D5F7F0780227D5E53
:10463F007F06801C7D0A7F0280167D327F028010EC
:10464F007D467F02800A7D0A7F038004AD4FE4FF21
:0E465F001276F7054E809EC26BAF4D125A4781
:01466D00222A
:1077740030290F900671E0FF7C0B7D101272E8B285
:107784002922202912900670E0FF7C0A7DF01272F3
:08779400E8B229E4786CF6224A
:10600F007D3F7F091276F77D507F081276F790005B
:10601F000EE493FDE4FF1276F77D5B7F061276F7B1
:10602F0090000FE493FDE4FF1276F7900010E493D5
:10603F00FDE4FF1276F7900011E49324BFB408003B
:10604F00505390605F75F003A4C58325F0C583732B
:10605F0002607702607B02607F02608502608B02C4
:10606F00609102609702609D7D0A80067D328002FA
:10607F007D467F02801C7D0A7F0380167D287F036B
:10608F0080107D467F03800A7D0A7F0480047D286F
:06609F007F041276F722D7
:1077EC008F53D26B125A477D4B7F021276F77D0472
:1077FC00E4FF1276F77D387F041276F712600FC221
:07780C006BAF53125A472233
:0B79AC00855182855083E0FFA3E0FDC1
:1079B700BF0A02E4FFBD0A02E4FDEF75F00AA42D39
:0279C700FF229D
:10534900C267D208D2207FF47E01127A1E7D2E7F99
:10535900031276F77D607F021276F7C208C2201227
:1053690033467F0812758740030254153049F012FD
:1053790033462049FA7868E6640770427E007F70F8
:1053890075331B7534108F828E837407F07D01E5A8
:10539900342DF582E43533F583E58224FFF582E582
:1053A9008334FFF583E0F9EF2DF582E43EF583E9D7
:1053B900F00DBD08DAD2677F647E00127A1E7F087D
:1053C900127587504720670302534BD208D2207FBA
:1053D900F47E01127A1E7D607F021276F77D327F9C
:1053E900061276F77D1E7F051276F7C208C2207C69
:1053F900007D707B087F787E001267C77F08127571
:105409008750097F327E00127A1E80F0126D3E7F2E
:06541900647E00127A1E01
:01541F00226A
:10774B00E4F53DC258C258F532302F05C22FC23F67
:10775B0022303005C230C24122303105C231C24322
:09776B0022303204C232C2452270
:104220007580FFC286E580540FFFC285E580C454C7
:10423000F04FF520D2867D027F0112625140107D41
:10424000037F011262514007300004D23980287D7B
:10425000027F01126251500A300007300104D23946
:1042600080157D037F01126251500A200003300146
:1042700004D2398002C2397D027F0212625140109D
:104280007D037F021262514007300204D23A802837
:104290007D027F02126251500A300207300304D2BD
:1042A0003A80157D037F02126251500A20020330CA
:1042B0000304D23A8002C23A7D027F031262514067
:1042C000107D037F031262514007300404D23B800B
:1042D000287D027F03126251500A30040730050422
:1042E000D23B80157D037F03126251500A200403E4
:1042F000300504D23B8002C23B7D027F0412625132
:10430000400F7D037F041262514006300603D23C09
:10431000227D027F041262515009300606300703E5
:10432000D23C227D037F04126251500920060330E3
:074330000703D23C22C23C4E
:014337002263
:10334600202B6EC25A20391C205019901CFAE070AE
:1033560002A3E0700B7D067F011262515002D24734
:10336600C249804D30392130501E901CE0E0700279
:10337600A3E0700B7D087F011262515002D23D30EE
:103386006502D25BD2498029303908205005126D7A
:103396003E801E20391B305018D25AC249C250C234
:1033A60014C210C21CC2181278F07868E66002D205
:1033B6005B202C71203A1C205319901CFCE07002F3
:1033C600A3E0700B7D067F021262515002D24BC2FF
:1033D6004D8052303A28305325901CE2E07002A30B
:1033E600E070127D087F0212625150097F02127846
:1033F600135002D23E306602D25BD24D8027303A5D
:1034060008205305126D92801C203A19305316C2BB
:103416004DC253C215C211C21DC219127A6D786906
:10342600E66002D25C202D71203B1C205519901CB1
:10343600FEE07002A3E0700B7D067F03126251501E
:1034460002D24EC2518052303B28305525901CE4A2
:10345600E07002A3E070127D087F031262515009EA
:103466007F031278135002D240302802D25BD25129
:103476008027303B08205505126DE6801C203B193D
:10348600305516C251C255C216C212C21EC21A12F7
:103496007A85786AE66002D25D202E6D203C1B207C
:1034A6005618901D00E07002A3E0700B7D067F04A5
:1034B6001262515002D252C25422303C2730562456
:1034C600901CE6E07002A3E070127D087F04126291
:1034D6005150097F041278135002D242302A02D288
:1034E6005BD25422303C06205603026E3A203C1929
:1034F600305616C254C256C217C213C21FC21B127E
:0A3506007A9D786BE66002D2602225
:047BBB0012508D22B5
:10508D0090001FE0540FFFBF010B304906203D0378
:10509D00025154C322EF64037014304906203D03BE
:1050AD00025154304D06203E0302515FC322EF647E
:1050BD00057014304906203D03025154305106202D
:1050CD00400302516AC322EF640970133049052071
:1050DD003D028073305406204203025175C322EF06
:1050ED006407701A304905203D02805B304D052064
:1050FD003E02805E3051052040028061C322EF6484
:10510D000B701A304905203D02803C304D05203E84
:10511D0002803F305405204202804DC322EF640DC2
:10512D00701A304905203D02801D30510520400286
:10513D00802B305405204202802EC322EF640F7065
:10514D002E304908203D05753E01D322304D0820F3
:10515D003E05753E02D322305108204005753E03B1
:10516D00D322305408204205753E04D322C322C3F6
:01517D00220F
:10781300BF010690001FE01322BF020790001FE084
:10782300A2E122BF030790001FE0A2E222BF0406E9
:0778330090001FE0A2E32218
:106D3E007868E6602275331B753410E4FFE5342F56
:106D4E00F582E43533F583E4F00FBF50F075331B55
:106D5E00753410E47868F6900600E0FFA3E0901C0E
:106D6E00E0CFF0A3EFF0900608E0FFA3E0901CFA4E
:106D7E00CFF0A3EFF0C246C247C25FC23DC265C2AA
:036D8E003FD250A1
:016D910022DF
:106D92007869E6602275351B753660E4FFE5362FAB
:106DA200F582E43535F583E4F00FBF50F075351BFD
:106DB200753660E47869F6900602E0FFA3E0901C65
:106DC200E2CFF0A3EFF090060AE0FFA3E0901CFCF4
:106DD200CFF0A3EFF0C248C24BC261C23EC266C24C
:036DE20041D25348
:016DE500228B
:106DE600786AE6602275371B7538B0E4FFE5382F00
:106DF600F582E43537F583E4F00FBF50F075371BA5
:106E06007538B0E4786AF6900604E0FFA3E0901CBB
:106E1600E4CFF0A3EFF090060CE0FFA3E0901CFE99
:106E2600CFF0A3EFF0C24CC24EC262C240C228C22B
:036E360043D255EF
:016E39002236
:106E3A00786BE6602275391C753A00E4FFE53A2F53
:106E4A00F582E43539F583E4F00FBF50F075391C4B
:106E5A00753A00E4786BF6900606E0FFA3E0901C12
:106E6A00E6CFF0A3EFF090060EE0FFA3E0901D003E
:106E7A00CFF0A3EFF0C24FC252C263C242C22AC2CB
:036E8A0045D25698
:016E8D0022E2
:10599200C208C209C20EC20C127A02C267D25EE407
:1059A200F53D7FE87E03127A1EC298C2AF75567F1C
:1059B200755596755498755300785374FF1259743F
:1059C200E4FBFAF9F8C3125961504430983E1200D0
:1059D20006127B7DEF14601824F0602624C1600B50
:1059E20024F670287F06127BAB802112714A801C3C
:1059F2007F06127BAB127520127673127022D26769
:105A0200800A7F06127BAB126756D2673067AAE420
:105A1200786CF6D26B7F01125A477F01126BE87DD8
:105A2200467F021276F77D1E7F071276F77D147F7E
:105A3200081276F77D327F031276F7C26B7F01126E
:045A42005A47C25E9F
:015A4600223D
:10675600756701756500756620E4F5577F02127B43
:10676600ABE5672402F559AF67127BABE4F558E554
:10677600662558F582E43565F583E0FF127BABE5C7
:10678600662558F582E43565F583E02559F5590502
:1067960058E558C3948040D7AF59127BAB7F03129C
:1067A6007BAB127BB3EF64156016056774802566B4
:1067B600F566E43565F5650557E557C39435409CA0
:0167C60022B0
:10752000756701756500756620E4F557127646505B
:10753000077F06127BAB80057F15027BAB05677466
:10754000802566F566E43565F5650557E557C3940E
:037550003540D9EA
:017553002215
:10764600E4F558127BB374502558F582E4341CF5E2
:1076560083EFF00558E558C3948440E7127AE19029
:0C7666001CD2E0B50705127911D322C335
:0176720022F5
:10791100E4FF74522FF582E4341CF583E0FEE56642
:0F7921002FF582E43565F583EEF0000FBF80E3AC
:017930002234
:107AE100E4FFFE74502EF582E4341CF583E02FFF91
:047AF1000EBE82EF54
:017AF500226E
:10714A00E4F557F55D755CE0755B93755A04F5597E
:10715A00785974FF125974E4FBFAF9F8C3125961A9
:10716A0050253098EB1200068F58E55864046017D2
:10717A00AF5D055D74502FF582E4341CF583E55844
:07718A00F02557F55780C9FD
:0171910022DB
:04000600AF99C29854
:01000A0022D3
:087BAB003099FDC2998F992267
:077BB3003098FDAF99C29864
:017BBA0022A8
:105BAF0007010203040506070707060504030201A0
:105BBF0003010A0A03020A0A03030A0A03040A0A70
:105BCF00030307050303020503070A0A04024B0038
:105BDF00040438072E03024B0004043802055F004B
:105BEF000302055F000402055F000502055F000662
:105BFF0002055F000702055F000802055F0009024A
:105C0F00055F000A02055F000B02055F000C02052D
:105C1F005F000D02055F000E02055F000F02055FBA
:105C2F00001002055F001102055F001204072E0825
:105C3F00260640033204072E082606400253080C9E
:075C4F000A1D040000241BE4
:10001600C2AF9000207491F09000217481F090009E
:1000260022F0900023F09000247403F090002574D1
:10003600BFF09000267418F0900027740FF090001F
:10004600307409F0A37403F0E4A3F0A37410F0A3D2
:100056007403F0E4A3F0A37415F0A37403F0A3747F
:1000660015F0A37403F0E4A3F0A37410F0A37403D3
:10007600F0E4A3F0A37409F0A37403F0A37415F0DD
:10008600A37403F0A314F0A3741AF0A37403F0E4AA
:10009600A3F0A3F0A3F0A3741AF0A37403F0A314BF
:1000A600F0A37415F0A37403F0E4A3F0A3F0A3F097
:1000B6007E5B7FBF7C007D807B041272A77E5B7FA8
:1000C600C37C007D887B041272A77E5B7FC77C00A1
:1000D6007D907B041272A77E5B7FCB7C007D987B34
:1000E600041272A77E5B7FD37C007DA07B04127214
:1000F600A77E5B7FCF7C007DA87B041272A77E5B08
:100106007FD77C007DB07B041272A77E5B7FAF7CBD
:10011600007D707B081272A77E5B7FB77C007D78BE
:100126007B081272A77E5B7FDB7C037D807B0912D6
:1001360072A77E5B7FE47C037DA07B071272A77E9D
:100146005B7FEB7C037DC07B051272A77E5B7FF035
:100156007C037DE07B051272A77E5B7FF57C047DC8
:10016600007B051272A77E5B7FFA7C047D207B05EF
:100176001272A77E5B7FFF7C047D407B051272A70F
:100186007E5C7F047C047D607B051272A77E5C7FAB
:10019600097C047D807B051272A77E5C7F0E7C0441
:1001A6007DA07B051272A77E5C7F137C047DC07BDD
:1001B600051272A77E5C7F187C047DE07B051272B7
:1001C600A77E5C7F1D7C057D007B051272A77E5C89
:1001D6007F227C057D207B051272A77E5C7F277CB3
:1001E600057D407B051272A77E5C7F2C7C057D60B9
:1001F6007B051272A77E5C7F317C057D807B0512B4
:1002060072A77E5C7F367C057DA07B051272A77E79
:100216005C7F3B7C057DC07B091272A77E5C7F44B8
:100226007C057DE07B091272A7900600E4F0A374BA
:10023600B4F0900602E4F0A374B4F0900604E4F07F
:10024600A374B4F0900606E4F0A374B4F090061814
:100256007401F0A374E0F090061AE4F0A37478F049
:1002660090061EE4F0A3743CF09006087402F0A316
:100276007458F090060A7402F0A37458F090060CB5
:100286007402F0A37458F090060E7402F0A374582A
:10029600F09006107401F0A3742CF090061274020C
:1002A600F0A37458F09006147403F0A37484F090CD
:1002B60006167404F0A374B0F07407900620F0A339
:1002C600F0900622F0A3F090061C7402F0A3745876
:1002D600F0900630740AF09006317428F0900633D8
:1002E600740AF0900634F09006327405F07E5C7F56
:1002F6004D7C067D407B091272A790063D7417F06F
:1003060090063E740CF090063C7419F0E490063F9B
:10031600F090063B740CF09006527401F090073092
:100326007469F0A37411F09006537401F0900750AD
:100336007469F0A37410F09006547401F09007707D
:100346007469F0A37421F09006557401F09007903B
:100356007469F0A37420F09006567401F09007B00B
:100366007469F0A37431F09006577401F09007D0C9
:100376007469F0A37430F09006587401F09007F099
:100386007469F0A37441F09006597401F090081056
:100396007469F0A37440F090065A7401F090083026
:1003A6007462F0A37411F0A37432F0A37401F0A385
:1003B6007450F0A37410F090065B7401F09008502E
:1003C6007461F0A37420F0A37462F0A37411F0A317
:1003D6007432F0A37402F0A37450F0A37410F0907A
:1003E600065C7401F09008707451F0A37411F0A3C8
:1003F6007433F0A3E4F0A37451F0A37410F09006E4
:100406005D7401F09008907462F0A37411F0A37407
:1004160030F0A37402F0A37462F0A37410F0900697
:100426005E7401F09008B07451F0A37411F0A374D7
:1004360041F0A37410F0A37451F0A37410F0900669
:100446005F7401F09008D07451F0A37411F0A37496
:1004560034F0A37414F0A37451F0A37410F0900652
:10046600607401F09008F07451F0A37411F0A37455
:1004760034F0A37418F0A37451F0A37410F090062E
:10048600617401F09009107451F0A37411F0A37413
:1004960034F0A37428F0A37451F0A37410F09006FE
:1004A600627401F09009307462F0A37411F0A374C1
:1004B60030F0A37403F0A37462F0A37410F09006F6
:1004C600637401F09009507462F0A37411F0A37480
:1004D60030F0A37404F0A37462F0A37410F09006D5
:1004E600647401F09009707462F0A37411F0A3743F
:1004F60060F0A37401F0A37495F0A3743DF0A374A7
:1005060090F0A37401F0A37498F0A37426F0A3747A
:1005160096F0A37440F0A37462F0A37410F0A37471
:1005260061F0A37470F09006657401F09009907400
:1005360062F0A37411F0A37460F0A37401F0A374C5
:1005460095F0A3743DF0A37490F0A37401F0A37426
:1005560096F0A37438F0A37462F0A37410F09006BA
:10056600667401F09009B07462F0A37411F0A3747C
:1005760060F0A37401F0A37495F0A3743DF0A37426
:1005860090F0A37402F0A37498F0A37426F0A374F9
:1005960096F0A37440F0A37462F0A37410F0A374F1
:1005A60061F0A37470F09006677401F09009D0743E
:1005B60062F0A37411F0A37460F0A37401F0A37445
:1005C60095F0A3743DF0A37490F0A37402F0A374A5
:1005D60096F0A37438F0A37462F0A37410F090063A
:1005E600687401F09009F07462F0A37411F0A374BA
:1005F60060F0A37401F0A37495F0A3743DF0A374A6
:1006060090F0A37403F0A37498F0A37426F0A37477
:1006160096F0A37440F0A37462F0A37410F0A37470
:1006260061F0A37470F09006697401F0900A10747A
:1006360062F0A37411F0A37460F0A37401F0A374C4
:1006460095F0A3743DF0A37490F0A37403F0A37423
:1006560096F0A37438F0A37462F0A37410F09006B9
:100666006A7401F0900A307462F0A37411F0A374F6
:1006760060F0A37401F0A37495F0A3743DF0A37425
:1006860090F0A37404F0A37498F0A37426F0A374F6
:1006960096F0A37440F0A37462F0A37410F0A374F0
:1006A60061F0A37470F090066B7401F0900A5074B8
:1006B60062F0A37411F0A37460F0A37401F0A37444
:1006C60095F0A3743DF0A37490F0A37404F0A374A2
:1006D60096F0A37438F0A37462F0A37410F0900639
:1006E6006C7401F0900A707462F0A37411F0A37434
:1006F60060F0A37401F0A37430F0A37405F0A37442
:1007060062F0A37410F090066D7401F0900A907474
:1007160062F0A37421F0A37460F0A37401F0A374D3
:1007260030F0A37406F0A37462F0A37420F0900670
:100736006E7401F0900AB07462F0A37431F0A37481
:1007460060F0A37401F0A37430F0A37407F0A374EF
:1007560062F0A37430F090066F7401F0900AD074C2
:1007660062F0A37441F0A37460F0A37401F0A37463
:1007760030F0A37408F0A37462F0A37440F09006FE
:10078600707401F0900AF07464F0A37411F0A3740D
:1007960096F0A37432F0A37495F0A3741EF0A374BC
:1007A60098F0A3744BF0A37464F0A37410F0900651
:1007B600717401F0900B107464F0A37411F0A374BB
:1007C60096F0A37432F0A37495F0A3741EF0A3748C
:1007D60093F0A37418F0A37464F0A37410F0900659
:1007E600737401F0900B507462F0A37411F0A3744B
:1007F60060F0A37401F0A37495F0A3743DF0A374A4
:1008060090F0A37402F0A37497F0A37426F0A37477
:1008160093F0A37418F0A37462F0A37410F0A37499
:1008260070F0A37410F09006747401F0900B70745D
:1008360062F0A37411F0A37460F0A37401F0A374C2
:1008460095F0A3743DF0A37490F0A37403F0A37421
:1008560097F0A37426F0A37493F0A37418F0A3740E
:1008660062F0A37410F0A37470F0A37420F09006E5
:10087600757401F0900B907462F0A37411F0A37478
:1008860060F0A37401F0A37495F0A3743DF0A37413
:1008960090F0A37404F0A37497F0A37426F0A374E5
:1008A60093F0A37418F0A37462F0A37410F0A37409
:1008B60070F0A37430F09006817401F0900D1074FE
:1008C60062F0A37411F0A37460F0A37401F0A37432
:1008D60092F0A3744BF0A37490F0A37404F0A37485
:1008E60094F0A37438F07499A3F0A3F0A37460F0A5
:1008F600A37401F0A37462F0A37410F01222F8122C
:100906007022D26B7F01125A477D2F7F071276F72E
:100916007D0C7F031276F77D327F061276F77D1EF9
:100926007F051276F790001F7401F0FD7F1F7E0091
:0B093600127328C26B7F01125A472287
:1022F8009001007402F0A3740DF0A37402F090062C
:10230800A014F09010F07464F0A37411F0A3749703
:10231800F0A3742EF0A37495F0A3743DF0A3749009
:10232800F0A37402F0A37496F0A37438F0A3746455
:10233800F0A37410F0A37470F0A37411F090010866
:102348007402F0A3740EF0A37402F09006A114F0C6
:102358009011107461F0A37410F0A37464F0A37466
:1023680011F0A37497F0A3742EF0A37495F0A374DE
:102378003DF0A37490F0A37402F0A37496F0A374D4
:1023880036F0A37464F0A37410F0A37470F0A3740F
:1023980010F09001107402F0A3740DF0A37403F010
:1023A8009006A27401F09011307464F0A37411F0D7
:1023B800A37497F0A3742EF0A37495F0A3743DF062
:1023C800A37490F0A37403F0A37496F0A37438F088
:1023D800A37464F0A37410F0A37470F0A37421F0D4
:1023E8009001187402F0A3740EF0A37403F0900621
:1023F800A37401F09011507461F0A37410F0A374E9
:1024080064F0A37411F0A37497F0A3742EF0A3746E
:1024180095F0A3743DF0A37490F0A37403F0A37433
:1024280096F0A37436F0A37464F0A37410F0A37448
:1024380070F0A37420F09001207402F0A3740DF0E2
:10244800A37404F09006A47401F09011707464F001
:10245800A37411F0A37497F0A3742EF0A37495F0ED
:10246800A3743DF0A37490F0A37404F0A37496F0E1
:10247800A37438F0A37464F0A37410F0A37470F01C
:10248800A37431F09001287402F0A3740EF0A374C1
:1024980004F09006A57401F09011907461F0A37493
:1024A80010F0A37464F0A37411F0A37497F0A374EC
:1024B8002EF0A37495F0A3743DF0A37490F0A37468
:1024C80004F0A37496F0A37436F0A37464F0A374B4
:1024D80010F0A37470F0A37430F09001307403F01E
:1024E800A3740DF0A37402F0A304F09006A674017F
:1024F800F09011B07464F0A37411F0A37497F0A372
:10250800742EF0A37495F0A3743DF0A37490F0A317
:102518007402F0A37490F0A37403F0A37496F0A36C
:102528007438F0A37464F0A37410F0A37470F0A36B
:102538007441F09001387403F0A3740EF0A3740290
:10254800F0A304F09006A77401F09011D07461F024
:10255800A37410F0A37464F0A37411F0A37497F03B
:10256800A3742EF0A37495F0A3743DF0A37490F0B7
:10257800A37402F0A37490F0A37403F0A37496F00C
:10258800A37436F0A37464F0A37410F0A37470F00D
:10259800A37440F09001407404F0A3740DF0A37488
:1025A80002F0A304F0A304F09006A87401F09011BF
:1025B800F07464F0A37411F0A37497F0A3742EF070
:1025C800A37495F0A3743DF0A37490F0A37402F083
:1025D800A37490F0A37403F0A37490F0A37404F0B0
:1025E800A37496F0A37438F0A37464F0A37410F085
:1025F800A37470F0A37441F0A37470F0A37451F045
:102608009001487404F0A3740EF0A37402F0A304BC
:10261800F0A304F09006A97401F09012107461F010
:10262800A37410F0A37464F0A37411F0A37497F06A
:10263800A3742EF0A37495F0A3743DF0A37490F0E6
:10264800A37402F0A37490F0A37403F0A37490F041
:10265800A37404F0A37496F0A37436F0A37464F022
:10266800A37410F0A37470F0A37440F0A37470F016
:05267800A37450F022E4
:0A72A7008E4C8F4D8C4E8D4F8B5096
:1072B100E4F9C3E5506480F8E96480985028E9FF57
:1072C1003395E0FEE54D2FF582E54C3EF583E493E1
:1072D100FFE9FD3395E0FCE54F2DF582E54E3CF5E8
:0672E10083EFF00980CCF0
:0172E7002284
:107A5300D291C2A4C2A5C2A6C2A7007F05127ACB47
:097A630000127AB500D2A7D291FD
:017A6C0022F7
:10797000127A53EF20E0F9D291C2A4C2A5C2A6C2E6
:0E798000A7007F06127ACB0000D2A7D2912278
:10798E00127A53EF20E0F9D291C2A4C2A5C2A6C2C8
:0E799E00A7007F04127ACB0000D2A7D291225C
:046E8E008E528F533E
:106E9200AE04AF058E568F57D291C2A4C2A5C2A628
:106EA200C2A7007F03127ACBE552FF127ACBAF530F
:106EB200127ACBE4F554F555127AB5E5572555F516
:106EC20082E5563554F583EFF00555E55570020518
:0E6ED20054C39420E554940040DED2A7D29120
:016EE000228F
:086905008E5D8F5E8C5F8D60DA
:10690D00127A53EF20E0F9127970855D63855E642C
:10691D00D291C2A4C2A5C2A6C2A7007F02127ACB91
:10692D00E55FFF127ACBAF60127ACBE4F561F562C9
:10693D00E5642562F582E5633561F583E0FF127A42
:10694D00CB0562E56270020561C39420E561940098
:07695D0040DE00D2A7D29139
:016964002210
:0A67C7008E4C8F4D8C4E8D4F8B5081
:1067D100C2AF127970127A53EF20E0F9854E5285DB
:1067E1004F53D291C2A4C2A5C2A6C2A7007F021272
:1067F1007ACBE54CFF127ACBAF4D127ACBE4F5514F
:10680100AF50EF3395E0FEC3E5519FEE6480F8741D
:1068110080985014E5532551F582E43552F583E013
:10682100FF127ACB055180D800D2A7D29112798E6E
:02683100D2AFE4
:016833002242
:107328008E5B8F5C8D5DC2AF127970127A53EF203D
:10733800E0F9D291C2A4C2A5C2A6C2A7007F0212D8
:107348007ACBE55BFF127ACBAF5C127ACBAF5D12DA
:0E7358007ACB0000D2A7D29112798ED2AF224A
:04783A008E4C8F4D94
:10783E00D291C2A4C2A5C2A6C2A77F03127ACBE57B
:10784E004CFF127ACBAF4D127ACB127AB5D2A7D2A9
:01785E009198
:01785F002206
:10719200C2AF754E00754F20755000755120E4F551
:1071A2004CF54DAD4FAC4EAF51AE50126E8E7420B9
:1071B200254FF54FE4354EF54E74202551F551E437
:1071C2003550F550054DE54D7002054CC394D6E59A
:0771D2004C940040CED2AF47
:0171D9002293
:10702200C2AF755B00755C20755900755A20E4F596
:1070320057F558AD5AAC59AF5CAE5B126905742076
:10704200255AF55AE43559F5597420255CF55CE466
:10705200355BF55B0558E55870020557C394D6E5D4
:0A70620057940040CE12798ED2AF91
:01706C002201
:046F33008C4D8D4EA6
:106F3700EF6048D22BD22CD22DD22EE4F54F854EBE
:106F470082854D83E0FEA3E04E6028AF4FEF339577
:106F5700E0FEEF25E0FFEE33FEE54E2FF582E54D2F
:106F67001254F5926720670B054FC3E54F64809471
:0B6F77009040CBC22BC22CC22DC22EBA
:016F820022EC
:0472E8008C4D8D4EEE
:1072EC00EF6038E4F54F854E82854D83E0FEA3E0D8
:1072FC004E6028AF4FEF3395E0FEEF25E0FFEE3305
:10730C00FEE54E2FF582E54D1254F5926720670B82
:0B731C00054FC3E54F6480949040CB08
:017327002243
:0854F5003EF583E0FEA3E0FF99
:0454FD00AD07AC0645
:10550100C268780CEF088006A2E0CE13CE13D8F85B
:10551100540FF5507808AF05AE04EF088006A2E0FD
:10552100CE13CE13D8F8540FF5517804AF05AE045D
:10553100EF088006A2E0CE13CE13D8F8540FF5522F
:10554100ED540FF553E550607CB4010BAB53AD52F4
:10555100AF5112581C806EE550B4030BAB53AD52E2
:10556100AF51126A80805EE550B4040BAB53AD526B
:10557100AF51126ADB804EE550B4050BAB53AD520F
:10558100AF51123CEC803EE550B4060BAB53AD522B
:10559100AF5112180F802EE550B4070BAB53AD522B
:1055A100AF51125420801EE550B4080BAB53AD52DD
:1055B100AF51126EE1800EE550B40909AB53AD5203
:0755C100AF51127885A268CA
:0155C80022C0
:10581C008F548D558B56E554B40113900020E0FF46
:10582C00126A28900020EFF0FD7F200258B7E55453
:10583C00B40211900021126A22900021EFF0FD7F3A
:10584C00210258B7E554B40310900022126A22903A
:10585C000022EFF0FD7F228052E554B4041090003A
:10586C0023126A22900023EFF0FD7F23803DE55444
:10587C00B40510900024126A22900024EFF0FD7FF2
:10588C00248028E554B40610900025126A2290005A
:10589C0025EFF0FD7F258013E554B4071390002607
:1058AC00126A22900026EFF0FD7F267E00027328FC
:1058BC00E554B40816900027126A22900027EFF0E6
:0C58CC00FD7F277E0012732812767322E5
:066A2200E0FFAB56AD558C
:106A2800D269AC07BD01047E018033BD02047E0239
:106A3800802CBD03047E048025BD04047E08801ECE
:106A4800BD05047E108017BD06047E208010BD079A
:106A5800047E408009BD08047E808002C269BB01B3
:106A680005EE4204800BEB7006EEF452048002C27D
:076A780069306903AF04223D
:016A7F0022F4
:106A80008F548D558B56E554700BAD56AF55127B18
:106A90005DE4FD801EE554B4010BAD56AF55127B8D
:106AA0005D7D01800EE554B4020CAD56AF55127BEE
:106AB0005D7D02023861E554B4030AE555700612A3
:106AC0007265C25822E554B40410AD56AF55126732
:0B6AD000248F3F753D05E53D70FC2262
:106ADB008F548D558B56E5547036E555B40108E54A
:106AEB005614FF7D018026E555B40208E55614FFC8
:106AFB007D028019E555B40308E55614FF7D03802C
:106B0B000CE55564047022E55614FF7D040271DA1E
:106B1B00E554B40114E555D39400400DE5559405A7
:0A6B2B005007753D01E53D70FC22A6
:103CEC008B54EF7017BD0114E5547002C220E554DB
:103CFC0064016003023E58D220023E58EF7017BD9B
:103D0C000214E5547002C221E55464016003023EC2
:103D1C0058D221023E58EF7017BD0314E5547002BF
:103D2C00C222E55464016003023E58D222023E587E
:103D3C00EF7017BD0414E5547002C223E5546401FE
:103D4C006003023E58D223023E58EF701BBD05188B
:103D5C00E5547004C220C221E55464016003023EA4
:103D6C0058D220D221023E58EF701BBD0618E554E4
:103D7C007004C222C223E55464016003023E58D28F
:103D8C0022D223023E58BF0117BD0114E554700224
:103D9C00C224E55464016003023E58D224023E580A
:103DAC00BF0117BD0214E5547002C225E55464012D
:103DBC006003023E58D225023E58BF0116BD0313C4
:103DCC00E5547002C226E55464016003023E58D2E9
:103DDC00268079BF0113BD0410E5547002C227E59B
:103DEC005464017067D2278063BF0117BD0514E5C9
:103DFC00547004C224C225E5546401704FD224D2FD
:103E0C00258049BF0117BD0614E5547004C226C2B3
:103E1C0027E55464017035D226D227802FEF640138
:103E2C00702AED64097025E554B401047F018019F2
:103E3C00E554B402047F028010E554B403047F03FC
:103E4C008007E554B404057F04126BE87F327E00D2
:043E5C00127A1E2296
:10180F008F548D558B56E5547016AD56AF55127BD0
:10181F005D901D14EFF0901D14E0D3940050F7224B
:10182F00E554B40117E555B40112E5567002C2082C
:10183F00E55664016003021BB5D20822E554B401DA
:10184F0017E555B40212E5567002C209E556640158
:10185F006003021BB5D20922E554B40117E555B454
:10186F000312E5567002C20EE55664016003021BB7
:10187F00B5D20E22E554B40117E555B40412E5565E
:10188F007002C20CE55664016003021BB5D20C2234
:10189F00E554B4011BE555B40516E5567004C208AE
:1018AF00C209E55664016003021BB5D208D20922B2
:1018BF00E554B40118E555B40613E5567004C20E8D
:1018CF00C20CE55664016003021BB58024E5546425
:1018DF00017023E555B4071EE5567008C208C2090A
:1018EF00C20EC20CE55664016003021BB5D208D2CA
:1018FF0009D20ED20C22E554B4021DE555B40118DD
:10190F00E5567004C208C220E55664016003021B4D
:10191F00B5D208D220021AD5E554B4021DE555B44C
:10192F000218E5567004C209C221E556640160032E
:10193F00021BB5D209D221021A61E554B4021DE58A
:10194F0055B40318E5567004C20EC222E556640161
:10195F006003021BB5D20ED222021A85E554B402DF
:10196F001DE555B40418E5567004C20CC223E556A4
:10197F0064016003021BB5D20CD223021AA8E554EE
:10198F0064027026E55564057020E5567008C2089C
:10199F00C209C220C221E55664016003021BB5D201
:1019AF0008D209D220D221021AD5E554640270263A
:1019BF00E55564067020E5567008C20EC20CC222AF
:1019CF00C223E55664016003021BB5D20ED20CD2BE
:1019DF0022D223021A85E55464027035E555640757
:1019EF00702FE5567010C208C209C20EC20CC22079
:1019FF00C221C222C223E55664016003021BB5D285
:101A0F0008D209D20ED20CD220D221D222D22380D8
:101A1F0065E554B4031DE555B40118E5567004C2CD
:101A2F0008C224E55664016003021BB5D208D22414
:101A3F00021AD5E554B4031FE555B4021AE55670E2
:101A4F0004C209C225E55664016003021BB5D20921
:101A5F00D2257F02021B04E554B4031EE555B403DF
:101A6F0019E5567004C20EC226E5566401600302E2
:101A7F001BB5D20ED2267F03807BE554B4031EE53F
:101A8F0055B40419E5567004C20CC227E55664011B
:101A9F006003021BB5D20CD2277F048058E5546433
:101AAF00037027E55564057021E5567008C208C21A
:101ABF0009C224C225E55664016003021BB5D20892
:101ACF00D209D224D2257F01802BE55464037028DC
:101ADF00E55564067022E5567008C20EC20CC22688
:101AEF00C227E55664016003021BB5D20ED20CD299
:101AFF0026D2277F03026BE8E554B4040AE555B4F8
:101B0F000105AF56026663E554B4040AE555B40205
:101B1F0005AF5602689DE5546409701EE555B40182
:101B2F0019E5567003C20A22E556B40103D20A2200
:101B3F00E556640270707F058069E5546409701E74
:101B4F00E555B40219E5567003C20B22E556B401F0
:101B5F0003D20B22E5566402704C7F068045E55494
:101B6F006409701EE555B40319E5567003C20F22C0
:101B7F00E556B40103D20F22E556640270287F07A1
:101B8F008021E5546409701EE555B40419E55670BB
:101B9F0003C20D22E556B40103D20D22E556B4025D
:071BAF00057F081260A5226A
:10542000AC07EC60030254D6BD010CEB7009900090
:105430001FE054FDF0800DBD010ABB010790001F65
:10544000E04403F0BD020CEB700990001FE054FB38
:10545000F0800DBD020ABB010790001FE04405F07B
:10546000BD030CEB700990001FE054F7F0800DBDF8
:10547000030ABB010790001FE04409F0BD040CEBD8
:10548000700990001FE054F9F0800DBD040ABB01C3
:105490000790001FE04407F0BD050CEB7009900079
:1054A0001FE054F3F0800DBD050ABB010790001FFB
:1054B000E0440DF0BD060CEB700990001FE054F1C4
:1054C000F08025ED64067020EB6401701B90001FD6
:1054D000E0440FF08012BC010FED700CEB7004C2C1
:1054E000298005BB0102D22990001FE0FD7F1F7EAD
:0554F0000012732822E8
:106EE1008F548D558B56E554700C127B59744F2F6E
:106EF100F58274068020E554B4010C127B59744F5D
:106F01002FF58274068024E554B40210127B597463
:106F11009F2FF58274063EF583E4F022E554B40315
:106F210010127B59749F2FF58274063EF58374010C
:026F3100F0224C
:027885008F541E
:10788700AF057804EF08800123D8FD4BF555E55483
:10789700B40908E555B4990302600FAD55AF54120A
:0278A70076F772
:0178A90022BC
:10666300E545B40109BF0106D220D2088060E545A3
:10667300B40109EF7006C220C2088052E545B40296
:1066830009BF0106D221D2098044E545B40209EFCE
:106693007006C221C2098036E545B40309BF01066D
:1066A300D222D20E8028E545B40309EF7006C22238
:1066B300C20E801AE545B40409BF0106D223D20CE9
:1066C300800CE545B40407EF7004C223C20C127AB0
:0A66D30002AF3E126BE81279E622D6
:10689D00E545B40108BF0105D224D20822E545B46F
:1068AD000108EF7005C224C20822E545B40208BFF5
:1068BD000105D225D20922E545B40208EF7005C2C3
:1068CD0025C20922E545B40308BF0105D226D20E23
:1068DD0022E545B40308EF7005C226C20E22E54538
:1068ED00B40408BF0105D227D20C22E545B4040734
:0868FD00EF7004C227C20C2257
:047B5900AD56AF5521
:0D7B5D00EF75F00AA47C002DFFEC35F0FE62
:017B6A0022F8
:020941008F4DD8
:10094300C268E4F53DD25ED26B125A477D4B7F02FB
:100953001276F77D04E4FF1276F77D387F04127672
:10096300F77D607F021276F790061CE0FFA3E0900C
:100973001CE8CFF0A3EFF0C26BAF4D125A47E4F57A
:1009830046C208123346E54DB40106A24992678078
:100993001FE54DB40206A24D92678014E54DB403E2
:1009A30006A25192678009E54DB40404A2549267EC
:1009B300901CE8E07002A3E07005D268020F8B3050
:1009C30067C1123346E54DB40106A2499267801F01
:1009D300E54DB40206A24D92678014E54DB40306BB
:1009E300A25192678009E54DB40404A25492672092
:1009F30067D0E54DB4010A754E1B754F10786880BA
:100A03002BE54DB4020A754E1B754F607869801C47
:100A1300E54DB4030A754E1B754FB0786A800DE53A
:100A23004DB4040B754E1C754F00786BE6F550E51D
:100A330050D394005003020F85854F82854E83E087
:100A4300640B6003020F80A3E0FFB40A0AE550B40D
:100A53000205D268020F85EF64017032854F8285EB
:100A63004E83A3A3E064037025E550B40520854FAE
:100A730082854E83A3A3A3E0FFE54F2404F582E41C
:100A8300354EF583E0FDAB4D123FBA020F85854F1E
:100A930082854E83A3E0B40121854F82854E83A3D3
:100AA300A3E0B40415E550D39405400EAB4DAD4F10
:100AB300AC4EAF50123510020F85854F82854E83A1
:100AC300A3E064017032854F82854E83A3A3E06463
:100AD300057025E550B40520854F82854E83A3A379
:100AE300A3E0FFE54F2404F582E4354EF583E0FDF2
:100AF300AB4D126567020F85854F82854E83A3E058
:100B030064017032854F82854E83A3A3E06406702F
:100B130025E550B40520854F82854E83A3A3A3E02A
:100B2300FFE54F2404F582E4354EF583E0FDAB4D3C
:100B3300125C56020F85854F82854E83A3E0B40174
:100B430021854F82854E83A3A3E0B40715E550D3D7
:100B53009405400EAB4DAD4FAC4EAF50124CAB02B3
:100B63000F85854F82854E83A3E064017032854FE4
:100B730082854E83A3A3E064087025E550B4052065
:100B8300854F82854E83A3A3A3E0FFE54F2404F59D
:100B930082E4354EF583E0FDAB4D126B35020F85D4
:100BA300854F82854E83A3E0B40219854F82854E1B
:100BB30083A3A3E0B4080DE550B40308AF4D127648
:100BC300CB020F85854F82854E83A3E06402702498
:100BD300854F82854E83A3A3E0B40818E550B4047F
:100BE30013854F82854E83A3A3A3E0FFAD4D1277F8
:100BF300C4020F85854F82854E83A3E0B402198515
:100C03004F82854E83A3A3E0B4090DE550B40308D6
:100C1300AF4D12769F020F85854F82854E83A3E0E9
:100C230064027024854F82854E83A3A3E0B4091820
:100C3300E550B40413854F82854E83A3A3A3E0FF3D
:100C4300AD4D12779C020F85854F82854E83A3E0BD
:100C530064037036854F82854E83A3A3E0640A70D4
:100C630029E55064057023854F82854E83A3A3A392
:100C7300E0FFE54F2404F582E4354EF583E0FD12F1
:100C830079B7AD4D12575D020F85854F82854E832F
:100C9300A3E06403703E854F82854E83A3A3E06483
:100CA300017031E550D39405402A854F82854E83E8
:100CB300A3A3A3E0FFE54F2404F582E4354EF583B7
:100CC300E0FD1279B7854D55AB50AD4FAC4E124692
:100CD3006E020F85854F82854E83A3E064037036D1
:100CE300854F82854E83A3A3E064027029E5506497
:100CF300057023854F82854E83A3A3A3E0FFE54FB1
:100D03002404F582E4354EF583E0FD1279B7AD4D49
:100D13001270B8020F85854F82854E83A3E0B4031A
:100D230019854F82854E83A3A3E0B4030DE550B428
:100D33000308AF4D127366020F85854F82854E837C
:100D4300A3E0B40321854F82854E83A3A3E0B404BB
:100D530015E550D39403400EAB4DAD50AF4FAE4E9F
:100D6300125EDE020F85854F82854E83A3E0B403B6
:100D730019854F82854E83A3A3E0B4050DE550B4D6
:100D83000308AF4D127B6B020F85854F82854E831F
:100D9300A3E0B4031D854F82854E83A3A3E0B4066D
:100DA30011E550B4050CAD4DAF4FAE4E1273DF02DB
:100DB3000F85854F82854E83A3E064037024854F9E
:100DC30082854E83A3A3E0B40718E550B4041385CA
:100DD3004F82854E83A3A3A3E0FFAD4D1279310269
:100DE3000F85854F82854E83A3E0B4031D854F8213
:100DF300854E83A3A3E0B40811E550B4050CAD4DB3
:100E0300AF4FAE4E1275B9020F85854F82854E8363
:100E1300A3E064057022E550B4041D854F82854E1E
:100E230083A3A3E0FF854F82854E83A3A3A3E0FDA5
:100E3300AB4D122D80020F85854F82854E83A3E033
:100E4300B40524E54F2404F582E4354EF583E0B47C
:100E53000B15E550D39405400EAB4DAD50AF4FAEDF
:100E63004E12477E020F85854F82854E83A3E06431
:100E7300067022E550B4041D854F82854E83A3A3DB
:100E8300E0FF854F82854E83A3A3A3E0FDAB4D1204
:100E9300267D020F85854F82854E83A3E0B4062409
:100EA300E54F2404F582E4354EF583E0B40B15E5F4
:100EB30050D39405400EAB4DAD50AF4FAE4E1231F3
:100EC3005E020F85854F82854E83A3E064097022FD
:100ED300854F82854E83A3A3E0B40A16E550B4047C
:100EE30011854F82854E83A3A3A3E0FF12706D0289
:100EF3000F85854F82854E83A3E064097023854F58
:100F030082854E83A3A3E0B40117E550B404128590
:100F13004F82854E83A3A3A3E0FFAD4D1256998064
:100F230061854F82854E83A3E0B40920854F828576
:100F33004E83A3A3E0B40214E550D39404400DAB55
:100F430050AD4DAF4FAE4E1214648036854F82853F
:100F53004E83A3E064097025854F82854E83A3A346
:100F6300E0B40317E550B40412854F82854E83A382
:100F7300A3A3E0FFAD4D126F8380078000AF4D1236
:100F830079C9206803020986C258D26BAF4D125A41
:100F9300477D607F021276F77D327F031276F7C2B8
:0F0FA3006BAF4D125A47127022E4786CF6C25EA3
:010FB200221C
:083510008F518C528D538B5436
:10351800855382855283A3A3A3E0FF8D828C83E524
:1035280082240412671B8F55E555D394005003027B
:1035380036B1E555942940030236B1E55164067069
:103548004FD26BAF54125A477D527F051276F7AFB0
:1035580055124BA9E5532405F582E43552F583E06D
:10356800B40112749F2555F582E43406F58374017D
:10357800F07D38800F749F2555F582E43406F58375
:10358800E4F07D367F061276F7C26BAF54025A47D5
:10359800E5532406F582E43552F583E0640B6003B5
:1035A8000236B1E5532405F582E43552F583E0B4DB
:1035B8000110749F2555F582E43406F5837401F0F3
:1035C800800D749F2555F582E43406F583E4F0E414
:1035D800FFFEE5532407F582E43552F583E5822E94
:1035E800F582E43583F583E0B40B04AF0680040E5E
:1035F800BE08DFEF70030236B1C3940840030236F9
:10360800B175F008E555A424F8F582E5F03400F525
:1036180083EFF07E01EF2401FDE433FCEEC39DEC63
:103628006480F87480985036E5532406F582E435B2
:1036380052F583E5822EF582E43583F583E0FD7546
:10364800F008E555A424F8F582E5F03400F583E5A3
:10365800822EF582E43583F583EDF00E80B7E553CD
:103668002408F582E43552F583E5822FF582E435A6
:1036780083F583E0640B602DEF2408FEC3E5519EBB
:10368800F55175F0041258D8AEF0EE701CE55324CD
:1036980007FDE43552FC7E00ED2FFBEE3CFAAD55FC
:1036A8007F011239EAD26A8002C26AAF54127B9D46
:0136B80022EF
:1078CE008E5CF55DAF5BEF3395E0FEE5592FF582EB
:0878DE00E5583EF583A3E0FF2D
:0A78E600EFD3940940037F00222233
:0839EA008F568D578A588B5946
:1039F200755B01E4F55AAF5BEF3395E0FEE5592FB5
:103A0200F582E5583EF583E0FF640970651278E6B9
:103A1200755C008F5DAE5C7804EF08800633CE33B0
:103A2200CE92E0D8F81278CEEF425DAE5CAF5D7810
:103A320008EF08800633CE33CE92E0D8F88E5CF5DC
:103A42005DAF5BEF3395E0FEE5592FF582E5583E19
:103A5200F583A3A3E0FFE55BFD3395E0FCE5592D7B
:103A6200F582E5583CF583A3A3A3E0FD1279B702E2
:103A72003B05AF5BEF3395E0FEE5592FF582E55844
:103A82003EF583E0FF1278E6755C008F5DAE5C78F0
:103A920004EF08800633CE33CE92E0D8F81278CE07
:103AA200EF425DAE5CAF5D7804EF08800633CE3343
:103AB200CE92E0D8F88E5CF55DAF5BEF3395E0FE19
:103AC200E5592FF582E5583EF583A3A3E0FF12786E
:103AD200E6EF425DAE5CAF5D7804EF08800633CE60
:103AE20033CE92E0D8F88E5CF55DAF5BEF3395E0B4
:103AF200FEE5592FF582E5583EF583A3A3A3E0FF27
:103B02001278E6EF425DE556701EAF5AEF3395E04C
:103B1200FEEF25E0FFEE33FE75F020E557A424D03A
:103B2200F582E5F034068021E556B4012FAF5AEF55
:103B32003395E0FEEF25E0FFEE33FE75F020E5570A
:103B4200A424D0F582E5F03410F583E5822FF582C6
:103B5200E5833EF583E55CF0A3E55DF07404255B47
:103B6200F55B055AC3E55A6480949050030239F814
:013B72002230
:084CAB008F518C528D538B5484
:104CB300855382855283A3A3A3E0FF8D828C83E572
:104CC30082240412671B8F55E555D39400500302C9
:104CD3004D98E55594334003024D98E551640670B1
:104CE3004FD26BAF54125A477D527F051276F7AFFE
:104CF30055124BA9E5532405F582E43552F583E0BB
:104D0300B40112744F2555F582E43406F58374011A
:104D1300F07D38800F744F2555F582E43406F58312
:104D2300E4F07D367F061276F7C26BAF54025A4722
:104D3300E5532406F582E43552F583E0640B7055A0
:104D4300E5532405F582E43552F583E0B40110748C
:104D53004F2555F582E43406F5837401F0800D7414
:104D63004F2555F582E43406F583E4F074F92551B3
:104D7300F55175F0041258D8AFF0EF7014E55324D1
:104D830006FBE43552FAAD55E4FF1239EAD26A80E4
:104D93000DC26A8009C26BAF54125A47C26AAF543C
:034DA300127B9DE3
:014DA60022EA
:023FBA008B5129
:103FBC001267248F54E554D3940050030240FEE55D
:103FCC0054943340030240FED26BAF51125A477DDA
:103FDC00527F051276F7AF54124BA9749F2554F5F6
:103FEC0082E43406F583E060047D3880027D367F00
:103FFC00061276F77F2C7E01127A1E75F008E554B6
:10400C00A424F8F582E5F03400F583E0F55270074E
:10401C007D1B7F061276F77D577F021276F7E552ED
:10402C0070030240AF755301AF52EF3395E0FEEFD2
:10403C002401FFE43EFEAD53ED3395E0FCC3ED9F50
:10404C00EE6480F8EC6480985059AF53EF3395E0F0
:10405C00FE75F008E554A424F8F582E5F03400F57B
:10406C0083E5822FF582E5833EF583E0FFD3940947
:10407C0040051272208028AF53EF3395E0FE75F0A7
:10408C0008E554A424F8F582E5F03400F583E582C4
:10409C002FF582E5833EF583E0FDE4FF1276F7050C
:1040AC005380857F2C7E01127A1E75F020E554A476
:1040BC0024D0F582E5F03410F583E0FEA3E0FF9008
:1040CC000000EEF0A3EFF04E70077D1B7F0612761A
:1040DC00F77D0C7F031276F7900000E07002A3E0EE
:1040EC006009E55414FD7F01122F74C26BAF5102AD
:0940FC005A47C26AAF51127B9DC4
:014105002297
:042F74008F558D5692
:102F7800E4F557E555600302301FAF57EF3395E08E
:102F8800FEEF25E0FDEE33FCAF56EF3395E0FEEFA4
:102F98007805C333CE33CED8F924F0F58274063ED3
:102FA800F583E5822DF582E5833CF583E0FAA3E01D
:102FB800FB780CFFAE02088006A2E0CE13CE13D831
:102FC800F8540FF5587808AF03AE02EF088006A250
:102FD800E0CE13CE13D8F8540FF559AF56EF33950A
:102FE800E0FEEF7805C333CE33CED8F924F0F5826E
:102FF80074063EF583E5822DF582E5833CF583E092
:10300800FCA3E0FD7804FFAE04088006A2E0CE131E
:10301800CE13D8F80230C2E555640160030230CB04
:10302800AF57EF3395E0FEEF25E0FDEE33FCAF56EA
:10303800EF3395E0FEEF7805C333CE33CED8F924CD
:10304800F0F58274103EF583E5822DF582E5833C28
:10305800F583E0FAA3E0FB780CFFAE02088006A235
:10306800E0CE13CE13D8F8540FF5587808AF03AE56
:1030780002EF088006A2E0CE13CE13D8F8540FF55D
:1030880059AF56EF3395E0FEEF7805C333CE33CE14
:10309800D8F924F0F58274103EF583E5822DF58287
:1030A800E5833CF583E0FCA3E0FD7804FFAE04086B
:1030B8008006A2E0CE13CE13D8F8540FF55AED547B
:1030C8000FF55BE558700FE559700BE55A7007E589
:1030D8005B700302315DAD58E4FF1276F7AD59E439
:1030E800FF1276F7E55864097048855A5CAF5CFEB4
:1030F8007804EF08800633CE33CE92E0D8F8F55C3A
:10310800E55B425CE55CB4990B7D09E4FF1276F758
:103118007D098027E55C75F00A84F55DFDE4FF1202
:1031280076F7E55D75F00AA4FFC3E55C9FF55DFDE4
:103138008009AD5AE4FF1276F7AD5BE4FF1276F72B
:103148007FF47E01127A1E0557C3E557648094A068
:053158005003022F7B73
:01315D00224F
:025C56008B5170
:105C58001267248F52E552D394005003025CF2E598
:105C68005294334003025CF2D26BAF51125A477D13
:105C7800527F051276F7AF52124BA9744F2552F591
:105C880082E43406F583E060047D3880027D367F47
:105C9800061276F77F2C7E01127A1E7F2C7E011267
:105CA8007A1E75F020E552A424D0F582E5F034067A
:105CB800F583E0FEA3E0FF900000EEF0A3EFF04EC6
:105CC80070077D1B7F061276F77D0C7F031276F72F
:105CD800900000E07002A3E06009E55214FDE4FFC3
:105CE800122F74C26BAF51025A47C26AAF51127B6E
:015CF8009D0E
:015CF9002288
:026567008B5156
:10656900126724AD07EDD39400406BED9433506668
:10657900E4FCECFF3395E0FEEF25E0FFEE33FE751A
:10658900F020EDA424D0F582E5F03410F583E582FE
:106599002FF582E5833EF583E4F0A3F00CBC10D21D
:1065A900749F2DF582E43406F583E4F0FCECFF33A7
:1065B90095E0FE75F008EDA424F8F582E5F03400C5
:1065C900F583E5822FF582E5833EF583E4F00CBC83
:0D65D90008DBD26A8002C26AAF51127B9DBE
:0165E6002292
:026B35008B5182
:106B3700126724AD07EDD394004045ED94335040E0
:106B4700E4FCECFF3395E0FEEF25E0FFEE33FE7546
:106B5700F020EDA424D0F582E5F03406F583E58234
:106B67002FF582E5833EF583E4F0A3F00CBC10D249
:106B7700744F2DF582E43406F583E4F0D26A80027F
:076B8700C26AAF51127B9DB1
:016B8E0022E4
:107554002430F58274003EF583EDF0AF55EF33959A
:10756400E0FEE5522FF582E5513EF583A3A3E0FF4B
:10757400D3EF648094814008EF6480948A500122A0
:037584007F002263
:107B4600D3EF648094804008EF648094A1500122B2
:037B56007F00228B
:081464008E518F528D538B5401
:10146C008F828E83A3A3A3E014F55674FC2554F548
:10147C00546403600FE55464076009E554640B6021
:10148C0003021807C3E556648094805003021807C2
:10149C00E556648094884003021807E4F555AF566E
:1014AC00EF3395E0FEEF7803C333CE33CED8F92477
:1014BC0030F58274003EF583AF55EF3395E0FEE5D1
:1014CC00822FF582E5833EF583E4F00555E555B4AE
:1014DC0008CC755504E5546403705FAF55EF339534
:1014EC00E0FEE5522FF582E5513EF583E0FFE55530
:1014FC00FD3395E0FCE5522DF582E5513CF583A3D7
:10150C00E0FD126724127B46AD07AF56EF3395E032
:10151C00FEEF7803C333CE33CED8F9127554AD0732
:10152C00AF56EF3395E0FEEF7803C333CE33CED80E
:10153C00F92431F58274000217FEE5546407600348
:10154C00021639AF55EF3395E0FEE5522FF582E5E3
:10155C00513EF583E0FFE555FD3395E0FCE5522D5A
:10156C00F582E5513CF583A3E0FD126724127B461E
:10157C00AD07AF56EF3395E0FEEF7803C333CE33B0
:10158C00CED8F9127554AD07AF56EF3395E0FEEF98
:10159C007803C333CE33CED8F92431F58274003EB0
:1015AC00F583EDF0AF55EF3395E0FEE5522FF58264
:1015BC00E5513EF583A3127570AD07AF56EF339529
:1015CC00E0FEEF7803C333CE33CED8F91266DD12CA
:1015DC007B46AD07AF56EF3395E0FEEF7803C33390
:1015EC00CE33CED8F92433F58274003EF583EDF07A
:1015FC00AF55EF3395E0FEE5522FF582E5513EF500
:10160C0083E5822406F582E43583F583E0FF1275C9
:10161C0074AD07AF56EF3395E0FEEF7803C333CECE
:10162C0033CED8F92434F58274000217FEE55464E5
:10163C000B6003021807AF55EF3395E0FEE5522F10
:10164C00F582E5513EF583E0FFE555FD3395E0FC71
:10165C00E5522DF582E5513CF583A3E0FD1267249C
:10166C00127B46AD07AF56EF3395E0FEEF7803C320
:10167C0033CE33CED8F9127554AD07AF56EF339540
:10168C00E0FEEF7803C333CE33CED8F92431F582A4
:10169C0074003EF583EDF0AF55EF3395E0FEE55267
:1016AC002FF582E5513EF583A3127570AD07AF5649
:1016BC00EF3395E0FEEF7803C333CE33CED8F91277
:1016CC0066DD127B46AD07AF56EF3395E0FEEF7843
:1016DC0003C333CE33CED8F92433F58274003EF5F0
:1016EC0083EDF0AF55EF3395E0FEE5522FF582E533
:1016FC00513EF583E5822406F582E43583F583E0DB
:10170C00FF127574AD07AF56EF3395E0FEEF78031B
:10171C00C333CE33CED8F92434F58274003EF5832E
:10172C00EDF0AF55EF3395E0FEE5522FF582E55124
:10173C003EF583E5822407F582E43583F583E0FFEB
:10174C00127574AD07AF56EF3395E0FEEF7803C317
:10175C0033CE33CED8F92435F58274003EF583EDC3
:10176C00F0AF55EF3395E0FEE5522FF582E5513E93
:10177C00F583E5822408F582E43583F583E0FFE503
:10178C0055FD3395E0FCE5522DF582E5513CF58392
:10179C00E582240912671B127B46AD07AF56EF3367
:1017AC0095E0FEEF7803C333CE33CED8F92436F56B
:1017BC008274003EF583EDF0AF55EF3395E0FEE516
:1017CC00522FF582E5513EF583E582240AF582E439
:1017DC003583F583E0FF127574AD07AF56EF339583
:1017EC00E0FEEF7803C333CE33CED8F92437F5823D
:1017FC0074003EF583EDF0D26A8002C26AAF5312D8
:02180C007B9DC2
:01180E0022B7
:10706D00EF24FE601014601314601624037016D202
:10707D0008D2248010D209D225800AD20ED22680C1
:10708D0004D20CD2277FF47E01127A1E753D04E5E1
:10709D003D70FC7F647E00127A1EC224C225C2267A
:0B70AD00C227C208C209C20EC20C229A
:045699008D51AC077C
:10569D00C3EC64809481500302575CEC6480948960
:1056AD00400302575CE4F552AF51EF3395E0FEEF46
:1056BD007803C333CE33CED8F924E8F582741A3E7D
:1056CD00F583AF52EF3395E0FEE5822FF582E5834A
:1056DD003EF583E0FD74182FF582741D3EF583EDC4
:1056ED00F00552E552B408C0EC14FFAD511271DA59
:1056FD00D269AF51125AFB753D017F327E00127A8D
:10570D001EE53D70FCC269AF51125AFBE4F552E53E
:10571D0052FD3395E0FC74182DF582741D3CF58314
:10572D00E0FBAF51EF3395E0FEEF7803C333CE339B
:10573D00CED8F924E8F582741A3EF583E5822DF56D
:0F574D0082E5833CF583EBF00552E552B408C0CA
:01575C00222A
:046F83008D51AC0779
:106F8700D3EC64809480403CEC648094895035E471
:106F9700FDECFF3395E0FEEF7803C333CE33CED855
:106FA700F92428F58274003EF583EDFF3395E0FE62
:106FB700E5822FF582E5833EF583E4F00DBD08D128
:0B6FC700D26A8002C26AAF51127B9DAB
:016FD200229C
:04466E008C528D538A
:10467200D3EF648094805003024776EF6480949570
:104682004003024776EB648094875003024776EB3F
:10469200648094E44003024776EF3395E0FEEF78BE
:1046A20005C333CE33CED8F92460F58274033EAF0E
:1046B20082F5568F57EB24FBF558D3940250030230
:1046C2004776E55875F00384E5F06003024776E526
:1046D2005875F00384F55AC39410400302477605D7
:1046E20057E557AE567002055614F5828E83E55A89
:1046F200F074052553F553E43552F552E4F558E5C7
:1047020058C3955A506A855382855283E0F559B44D
:104712000A130557E557AE567002055614F5828EF8
:1047220083E4F080120557E557AE56700205561421
:10473200F5828E83E559F0855382855283A3E0FF8B
:10474200855382855283A3A3E0FD1279B78F590561
:1047520057E557AE567002055614F5828E83E55919
:10476200F074032553F553E43552F5520558808F02
:0B477200D26A8002C26AAF55127B9D24
:01477D002219
:04575D008F518D5289
:10576100E551D394005003025814E55194154003B8
:10577100025814D26BAF52125A477D5F7F051276E1
:10578100F7AD51E4FF1276F77D527F041276F77F71
:10579100F47E01127A1E75F020E551A42460F58291
:1057A100E5F03403AF82F5558F56F583E0F553608C
:1057B1004DD394004056E55394105050E55325E0E5
:1057C100F553755401E5532401FFE433FEC3E55459
:1057D1009FEE6480F87480985032E5562554F58226
:1057E100E43555F583E0FFE5562554F582E435555A
:1057F100F583A3E0FD1276F70554055480C77D1BA0
:105801007F061276F77D5F7F051276F7C26BAF5286
:0A581100025A47C26AAF52127B9D93
:01581B00226A
:10779C008D51EFD3940A4006EFD3940F4003EF7052
:1077AC000E90063FEFF0D26AAF51127B9DD322C2EE
:0877BC006AAF51127B9DC3224C
:1077C4008D51EFD3940A4006EFD3940F4003EF702A
:1077D4000E90063BEFF0D26AAF51127B9DD322C2CA
:0877E4006AAF51127B9DC32224
:107220008F55E555B40B067D5F7F078034E555B477
:107230000C067D5E7F068029E555B40D067D0A7F2C
:1072400002801EE555B40E067D327F028013E5559F
:10725000B40F067D467F028008E55570077D0A7FE2
:05726000031276F72285
:10769F008F51D26B125A477D207F051276F77D2EC0
:1076AF007F031276F77D527F041276F790063FE044
:0C76BF00FF127220C26BAF51125A47221A
:1076CB008F51D26B125A477D207F051276F77D21A1
:1076DB007F061276F77D527F041276F790063BE019
:0C76EB00FF127220C26BAF51125A4722EE
:107931008D51D3EF64809480400EEF648094865023
:10794100071274B8D26A8002C26AAF51127B9D22BB
:0673DF008D51AB07AA0668
:1073E5008B828A83A3A3A3E0FFEB2404F582E43A0E
:1073F500126720D3EF648094804010EF648094A1DD
:10740500500990063DEFF0D26A8002C26AAF511270
:027415007B9D5D
:017417002252
:0675B9008D51AB07AA068C
:1075BF008B828A83A3A3A3E0FFEB2404F582E43A32
:1075CF00126720EFC39421500990063CEFF0D26A66
:0975DF008002C26AAF51127B9DCB
:0175E8002280
:065EDE008E518F528B5320
:105EE400755406755540D3ED64809484407CED640C
:105EF4008094A55075ED24FDF556D39404406BE5CC
:105F04005620E06613F5570555E555AE5470020565
:105F14005414F5828E83E557F074032552F552E448
:105F24003551F551E4F556E556C39557503385522E
:105F340082855183E0FFA3E0FD1279B70555E5554D
:105F4400AC547002055414F5828C83EFF00552E5CD
:105F540052700205510552E55270020551055680F2
:105F6400C6D26AAF53127B9DD322C26AAF53127B4F
:025F74009DC3CB
:015F76002208
:08477E008E518F528D538B54B4
:10478600C269D3E553648094845003024833E553E9
:104796006480948D40030248338F828E83A3A3E006
:1047A600640A60030248338F828E83A3A3A3E014B6
:1047B600B4080050769047C975F003A4C58325F068
:1047C600C583730247E10247EB0247F50247FF0242
:1047D600480902481302481D0248277555007556B8
:1047E60080D2698048755500755688D269803E75B5
:1047F6005500755690D2698034755500755698D215
:1048060069802A7555007556A0D2698020755500B5
:104816007556A8D26980167555007556B0D269804E
:104826000C755500755678D2698002C26930695098
:10483600E4FFEF7C002556FDEC35558D82F583E4CB
:10484600F00FBF08EDE55324FB855682855583F0AE
:104856007F01E5522404F582E43551F583E5822F84
:10486600F582E43583F583E0FEEF7C002556FDEC0A
:1048760035558D82F583EEF00FBF08D6D26A8002D9
:07488600C26AAF54127B9DD2
:01488D002208
:0461C6008E548F550F
:1061CA000555E5557002055414F5828E83E0F5579E
:1061DA006074C39408506F7F2C7E01127A1EE4F516
:1061EA0056E556C39557505E855582855483E060BF
:1061FA003624F5601414601714601A14601D1460B4
:10620A002024057028E4FD802D7D5F7F0780287D8E
:10621A005E7F0680227D0A7F02801C7D327F02809B
:10622A00167D467F0280107D0A7F03800A8555828B
:10623A00855483E0FDE4FF1276F70555E5557002B3
:06624A0005540556809B7F
:01625000222B
:022D80008B5175
:102D8200C269EF640A6003022F5BED14B4080040CD
:102D920003022F59902DA475F003A4C58325F0C515
:102DA2008373022DBC022DF0022E24022E58022E15
:102DB2008C022EC0022EF3022F26D26BAF51125A72
:102DC200477D577F021276F77D05E4FF1276F7E41E
:102DD200FDFF1276F77D01E4FF1276F77D527F0444
:102DE2001276F7755200755380D269022F5BD26B4F
:102DF200AF51125A477D577F021276F77D05E4FFE5
:102E02001276F7E4FDFF1276F77D02E4FF1276F701
:102E12007D527F041276F7755200755388D269028B
:102E22002F5BD26BAF51125A477D577F021276F752
:102E32007D05E4FF1276F7E4FDFF1276F77D03E4E9
:102E4200FF1276F77D527F041276F77552007553A2
:102E520090D269022F5BD26BAF51125A477D577FD6
:102E6200021276F77D05E4FF1276F7E4FDFF127693
:102E7200F77D04E4FF1276F77D527F041276F77530
:102E82005200755398D269022F5BD26BAF51125A1E
:102E9200477D577F021276F77D05E4FF1276F7E44D
:102EA200FDFF1276F77D05E4FF1276F77D527F046F
:102EB2001276F77552007553A0D269022F5BD26B5E
:102EC200AF51125A477D577F021276F77D05E4FF14
:102ED2001276F7E4FDFF1276F77D06E4FF1276F72D
:102EE2007D527F041276F77552007553A8D269801D
:102EF20068D26BAF51125A477D577F021276F77D27
:102F020005E4FF1276F7E4FDFF1276F77D07E4FF92
:102F12001276F77D527F041276F77552007553B020
:102F2200D2698035D26BAF51125A477D577F021258
:102F320076F77D05E4FF1276F7E4FDFF1276F77D62
:102F420008E4FF1276F77D527F041276F77552007D
:102F5200755378D2698002C269306909AF53AE52A3
:102F62001261C68005AF511279C9C26BAF51125AB4
:012F72004717
:012F7300223B
:08315E008E518F528D538B54EA
:10316600C2698F828E83A3A3E0640A6003023215CC
:10317600124AA28E568F57D3E557943BE5569400D4
:103186005003023210E5579408E5569407507BC366
:10319600E5536480948A5072855282855183A3A335
:1031A600A3E0F555B401069006000232BBE555B41E
:1031B60002069006020232BBE555B40306900604E9
:1031C6000232BBE555B404069006060232BBE5554D
:1031D600B405069006080232BBE555B4060690060D
:1031E6000A0232BBE555B4070690060C0232BBE56F
:1031F60055B4080690060E0232BBE555B409069092
:1032060006100232BBD269023337D26902333785E0
:103216005282855183A3A3E0640160030232C5ADE7
:1032260053AF52AE51124AA28E568F57D3E55794DA
:103236003BE55694005003023337E5579408E556AC
:1032460094074003023337C3E5536480948A4003EE
:10325600023337855282855183A3A3A3E0F555B483
:103266000A05900612804EE555B4010590061480B5
:1032760044E555B40205900616803AE555B40305B3
:103286009006188030E555B4040590061A8026E5A8
:1032960055B4050590061C801CE555B40605900638
:1032A6001E8012E555B407059006208008E555B442
:1032B6000809900622E556F0A3806FD269807285D0
:1032C6005282855183A3A3E064027065AD53AF5269
:1032D600AE51126B8F7556008F57C3E5579463E551
:1032E600569400504CC3E5536480948850438552ED
:1032F60082855183A3A3A3E0F555B4010790063058
:10330600EFF0802DE555B40205900631801CE55599
:10331600B403059006328012E555B40405900633D1
:103326008008E555B40508900634E557F08002D2CA
:0F33360069306904C26A8002D26AAF54127B9D6B
:013345002265
:10267D008F518D528B53E551640A6003022729E572
:10268D0052C3940A40030228FFD26BAF53125A472C
:10269D007D277F081276F77D06E4FF1276F7E4FDBD
:1026AD00FF1276F7AD52E4FF1276F77D527F0412DA
:1026BD0076F7E55214B4090040030228F89026D8A5
:1026CD0075F003A4C58325F0C583730226F3022696
:1026DD00F90226FF02270502270B022711022717F1
:1026ED0002271D02272390060002283990060202B8
:1026FD0028399006040228399006060228399006DA
:10270D000802283990060A02283990060C02283949
:10271D0090060E022839900610022839E551640101
:10272D006003022847E552D394004006E552940910
:10273D004009E552640A6003022844D26BAF53127C
:10274D005A477D277F081276F77D06E4FF1276F74C
:10275D00E552B40A147D0AE4FF1276F77D527F0428
:10276D001276F7900612022839E552B401147D0B4A
:10277D00E4FF1276F77D527F041276F7900614026D
:10278D002839E552B402147D0CE4FF1276F77D5220
:10279D007F041276F7900616022839E552B403131A
:1027AD007D0DE4FF1276F77D527F041276F79006C9
:1027BD00188079E552B404137D0EE4FF1276F77D8F
:1027CD00527F041276F790061A8061E552B4051314
:1027DD007D0FE4FF1276F77D527F041276F7900697
:1027ED001C8049E552B406137D10E4FF1276F77D87
:1027FD00527F041276F790061E8031E552B407130E
:10280D007D11E4FF1276F77D527F041276F7900664
:10281D00208019E552640860030229067D12FF121B
:10282D0076F77D527F041276F7900622E0FEA3E044
:10283D00FF1274830229060228FFE551640260032A
:10284D00022906E552D3940050030228FFE5529465
:10285D000740030228FFD26BAF53125A477D277FE3
:10286D00081276F77D06E4FF1276F77D14E4FF1269
:10287D0076F7E55224FE6020146030146040146039
:10288D0050240470667D01E4FF1276F77D527F04BB
:10289D001276F7900630804A7D02E4FF1276F77DBE
:1028AD00527F041276F790063180377D03E4FF12D4
:1028BD0076F77D527F041276F790063280247D04E0
:1028CD00E4FF1276F77D527F041276F7900633807F
:1028DD00117D05E4FF1276F77D527F041276F79095
:1028ED000634E0FF7E001275E9800EAF531279C9F0
:1028FD008007C26AAF53127B9DC26BAF53125A470A
:01290D0022A7
:064AA2008E588F59A90592
:104AA8007D057C00E5592DF582E5583CF583E0C38A
:104AB800940A400CE5592DF582E5583CF583E4F05D
:104AC8000DBD00010CED640A4C70D9B90610E5590A
:104AD8002405F582E43558F583E0FF7E0022E96479
:104AE800077019E5592405F582E43558F583E07512
:104AF800F00AA4ACF0FDE55924068032E964087098
:104B08003DE5592405F582E43558F583E075F064F0
:104B1800A4ACF0FDE5592406F582E43558F583E0A8
:104B280075F00AA42DFDE5F03CFCE5592407F58253
:104B3800E43558F583E02DFDE43CAF05FE22E96439
:104B480009705AE5592405F582E43558F583E0FFE4
:104B58007E007C037DE81258FAAC06AD07E55924BF
:104B680006F582E43558F583E075F064A42DFDE57B
:104B7800F03CFCE5592407F582E43558F583E075E7
:104B8800F00AA42DFDE5F03CFCE5592408F582E483
:104B98003558F583E02DFDE43CFEAF0522E4FEFF29
:014BA80022EA
:066B8F008E588F59A90584
:106B95007F057E00E5592FF582E5583EF583E0C374
:106BA500940A400CE5592FF582E5583EF583E4F04B
:106BB5000FBF00010EEF64084E70D9E9640770201D
:106BC500E5592405F582E43558F583E075F00AA406
:106BD500FFE5592406F582E43558F583E02FFF22B9
:026BE5007F002F
:016BE700228B
:104BA9008F56E556D3945940147D5AE4FF1276F78F
:104BB900E55624A6FD7003024CAA024CA5E556D37E
:104BC900944F401AE556945A50147D50E4FF1276DA
:104BD900F7E55624B0FD7003024CAA024CA5E55630
:104BE900D39445401AE556945050147D46E4FF127B
:104BF90076F7E55624BAFD7003024CAA024CA5E5E6
:104C090056D3943B4019E556944650137D3CE4FF36
:104C19001276F7E55624C4FD7003024CAA807DE59F
:104C290056D394314016E556943C50107D32E4FF3A
:104C39001276F7E55624CEFD60678060E556D39479
:104C4900274016E556943250107D28E4FF1276F776
:104C5900E55624D8FD604A8043E556D3941D401695
:104C6900E556942850107D1EE4FF1276F7E5562488
:104C7900E2FD602D8026E556D394134016E556943F
:104C89001E50107D14E4FF1276F7E55624ECFD6002
:104C9900108009E556C394145007AD56E4FF127607
:024CA900F722F0
:1075E9008E548F557C007D0A12590CAD07E4FF12A9
:1075F90076F77D5B7F061276F7AE54AF557C007D3A
:107609000A12590CE4FF1276F77D4A7F070276F7D2
:047483008E548F553F
:107487007C007D3C12590CAA06AB07124BA97D055F
:107497007F061276F7AE54AF557C007D3C12590C2F
:1074A700ED4C600CAF05124BA97D4A7F071276F7AA
:0174B70022B2
:0270B8008D51F8
:1070BA00D3EF648094804038EF648094955031EF28
:1070CA003395E0FEEF7805C333CE33CED8F924608A
:1070DA00F58274033EAF82FEE4FD0FEFAA0670014B
:1070EA000E14F5828A83E4F00DBD20EED26A800286
:0770FA00C26AAF51127B9D39
:01710100226B
:107366008F51900640E0D394024015D269125AFB21
:10737600753D037F327E00127A1EE53D70FC801556
:10738600D269AF51125AFB7D1B7F061276F77D0C30
:0D7396007F031276F7C269AF51125AFB2235
:107B6B007E10900640E4F0A3DEFC7E10D26A127BFE
:017B7B009D6C
:017B7C0022E6
:1078AA008F5CD26B125A477D607F021276F77D3267
:1078BA007F061276F77D1E7F051276F7C26BAF5CE4
:0478CA00125A4722E5
:1079C9008F5CD26B125A477D607F021276F77D3049
:0D79D9007F031276F7C26BAF5C125A472293
:0E7B9D008F5B306A030278AAAF5B1279C922AF
:1066DD002432F58274003EF583EDF0AF55EF33951E
:1066ED00E0FEE5522FF582E5513EF583E582240467
:1066FD00F582E43583F583E0FFE555FD3395E0FC48
:10670D00E5522DF582E5513CF583E5822405F582B0
:07671D00E43583F583E0FD84
:10672400EFD394004015EF940B5010EFC3940A502C
:1067340008EF75F00AA4FE8002E4FEEDD394004055
:106744000EED940B5009EDC3940A5003ED2EFEAFE9
:01675400063E
:016755002221
:03000000027B8EF2
:0F7B8E00758E0078FEE4F6D8FD75816C02517E8D
:107AB500D292C0F075F008C29100A29233D291D54E
:067AC500F0F5D0F0FF22F5
:107ACB00EFC0F075F00833C291929333D291D5F099
:067ADB00F6D0F0C291227A
:1076F700EFFEEDFF1280008E2F8F30125CFA755F60
:1077070064AF5F155FEFD39400400EE4F55EE55E6E
:09771700C3943A50EC055E80F5C4
:017720002246
:105CFA00D2A885A86175A881C244853082852F8380
:105D0A00E493F560C4540FF5604360F0856080C287
:105D1A0084D28500C2870000D287007580FF758013
:105D2A00FEC284C28500C28700000000D2870075C7
:105D3A0080FFD24475623E756380E4F56030941D3D
:105D4A000560E560B464F6123346E56315637002D4
:105D5A001562D3E5639400E562940050DD75623EF6
:105D6A00756380E4F56020941D0560E560B464F60F
:105D7A00123346E563156370021562D3E563940036
:105D8A00E562940050DD8561A8C2A87F147E0012E6
:025D9A007A1E6F
:015D9C0022E4
:107721007580FDC284C28500C28700000000D28737
:10773100007580FF7F147E00127A1E7F997E0912E8
:0A77410080008E2F8F30125CFA22B8
:1058D800C2D530F707B2D563F0FF05F030E70CB258
:1058E800D5F4048463F0FF05F080018430D502F418
:0258F800042288
:1058FA00EF8DF0A4A8F0CF8CF0A428CE8DF0A42EC2
:02590A00FE227B
:10590C00BC000BBE0029EF8DF084FFADF022E4CC7F
:10591C00F875F008EF2FFFEE33FEEC33FCEE9DEC48
:10592C00984005FCEE9DFE0FD5F0E9E4CEFD22ED8E
:10593C00F8F5F0EE8420D21CFEADF075F008EF2FD8
:10594C00FFED33FD4007985006D5F0F222C398FDC9
:05595C000FD5F0EA2266
:10596100EB9FF5F0EA9E42F0E99D42F0E89C45F09C
:015971002213
:105972007401FF3395E0FEFDFC080808E6CF2FF620
:1059820018E6CE3EF618E6CD3DF618E6CC3CF622F9
:107B7D00EFC39461400AEF947B5005EF24E0FF22A0
:017B8D0022D5
:00000001FF
